:10000000300A01202506000021060000210600001C
:10001000210600002106000021060000000000006B
:1000200000000000000000000000000021060000A9
:10003000210600000000000021060000210600004B
:100040002106000021060000210600002106000014
:100050002106000021060000210600002106000004
:1000600021060000210600002106000021060000F4
:1000700021060000210600002106000021060000E4
:1000800021060000210600002106000021060000D4
:1000900021060000210600002106000021060000C4
:1000A00021060000210600002106000021060000B4
:1000B00021060000210600002106000021060000A4
:1000C0002106000021060000210600002106000094
:1000D0002106000021060000210600002106000084
:1000E00021060000210600000000000000000000C2
:1000F00000000000E90500002106000021060000C4
:100100002106000021060000210600002106000053
:100110002106000021060000210600002106000043
:100120002106000021060000210600002106000033
:100130002106000021060000210600002106000023
:100140002106000021060000210600002106000013
:100150002106000021060000210600002106000003
:1001600021060000210600002106000021060000F3
:1001700021060000210600002106000021060000E3
:1001800021060000210600002106000021060000D3
:1001900021060000210600002106000021060000C3
:1001A00021060000210600002106000021060000B3
:1001B00021060000210600002106000021060000A3
:1001C0002106000021060000210600002106000093
:1001D0002106000021060000210600002106000083
:1001E0002106000021060000210600002106000073
:1001F0002106000021060000210600002106000063
:100200002106000021060000210600002106000052
:100210002106000021060000210600002106000042
:100220002106000021060000210600002106000032
:100230002106000021060000210600002106000022
:100240002106000021060000210600002106000012
:100250002106000021060000210600002106000002
:10026000210600000348044B834202D0034B03B134
:1002700018477047A8880000A88800000000000008
:100280000548064B1B1AD90F01EBA301491002D0F8
:10029000034B03B118477047A8880000A8880000E6
:1002A0000000000010B5064C237843B9FFF7DAFFD1
:1002B000044B13B10448AFF300800123237010BD39
:1002C0009C09002000000000A888000008B5044B2D
:1002D0001BB104490448AFF30080BDE80840CFE7F4
:1002E00000000000A0090020A888000070B50D469D
:1002F0001646044610B1081E18BF01200549064BDA
:10030000342298472368324629462046BDE870408B
:10031000184700BF4C83000079040000044A1168AC
:10032000034609B90349116010680344136070471C
:10033000B8090020300A01204FF0FF3070474FF419
:1003400000534B6000207047012070470020704729
:1003500008B50146014B02489847FEE739190000ED
:100360006083000070474FF0FF3070471FB503896E
:10037000ADF804304FF40043ADF806300391054B5F
:10038000029201A9143814469847002808BF204655
:1003900004B010BDE10C00001FB50389ADF80430B6
:1003A00048F20103ADF806300391054B029201A912
:1003B000143814469847002808BF204604B010BDE2
:1003C000E10C000038B50446003818BF0120074B87
:1003D0000D465E2206499847064B29462046984717
:1003E00018B9054BA361054B636138BD7904000062
:1003F000798300008D0C0000990300006D0300005C
:10040000004B1847B90C000002F48062C1F30901E7
:100410001143818308467047094A138810B59BB27F
:100420001380084B9847084B9847084B9847084B50
:100430009847BDE81040074B40F6FF70184700BFD3
:10044000004000410507000081040000DD050000B8
:100450009904000059040000C30707D5044B054A5E
:100460001A6243F6FD7259681142FCD1704700BF11
:10047000001C00400101010000B900BE70470000EF
:10048000034B044A9A611A699207FCD5704700BF72
:100490000010004006260003704700002DE9F843D5
:1004A0000E461546044618B129B3101E18BF012088
:1004B0001249134BDFF85080F12298470834204648
:1004C000C0470028FBD0DFF844900027F15D2046AC
:1004D000C8472046C0470028FBD00137BD42F5D8A9
:1004E000002D084E08BF01252046B0470028FBD04C
:1004F0002846BDE8F8830846DAE700BF9583000088
:1005000079040000790C00006F0C0000610C000001
:100510002DE9F8430E461546044618B1E9B1101E00
:1005200018BF01200E490F4BDFF83C90DFF83C80EC
:100530004FF486729847002708342046C8470028A1
:10054000FBD02046C047F0550137BD42F5D8002DFD
:1005500014BF28460120BDE8F8830846E2E700BF43
:100560009583000079040000830C0000670C0000F4
:1005700038B50D46044610B1081E18BF01200749C2
:10058000074B34229847074B294604F10800984747
:1005900018B9054B6360054B236038BD9583000097
:1005A000790400002D0C0000110500009D040000DE
:1005B00010B50446003818BF01200549054B5322E9
:1005C000984704F10800044B9847002010BD00BF75
:1005D0009583000079040000550C0000014B0122B6
:1005E0005A717047000800400B4A937882B0DBB222
:1005F0000193019B990705D5084B1B6813B15068FF
:1006000002B01847019BDB0704D5044B5B680BB1B4
:10061000014AF4E702B0704700000241BC09002023
:10062000FEE7000018491948814210B50AD0184B5E
:10063000DA1C121A22F00302C41EA34238BF0022A1
:10064000144B9847144B1548DA1C121AC11E22F09D
:100650000302994288BF0022114B00219847114A9A
:10066000114B22F07F029A60D3F8882042F4700286
:10067000C3F88820BFF34F8FBFF36F8F0B4B9847A2
:100680000B4B9847FEE700BFA88800000000002041
:100690009C09002061170000300A00209C090020FE
:1006A000951800000000000000ED00E019170000A0
:1006B000B506000008B50A4B0A4C98470A4B984704
:1006C0000A4B98470A48A0471B210A48A0471B210C
:1006D0000948A04709481B21A047094B9847FEE756
:1006E0004D0E0000650E0000550E0000CD0E0000FE
:1006F000B1830000C9830000CF830000D4830000D1
:10070000F10E0000034BDA6902F47C52DA61012237
:100710001A747047001400404309DB0103F182435F
:1007200030B503F5004300F01F041D1903EB54031B
:1007300095F8402002F0FE0242F0010285F84020C8
:1007400093F8302010F0010FC9B21BBF02F00F0266
:1007500042EA011202F0F002D2B20ABF114383F85A
:10076000302083F8301030BD10B5054C05493920D4
:10077000A04723460449BDE810403820184700BF71
:10078000190700000300390003003800064B40221F
:10079000C3F8DC204322C3F88C20044A936943F455
:1007A00000739361704700BF001C004000080040C8
:1007B00010B5054B054906489847064B0022984757
:1007C000BDE81040044B18478D0700000020014190
:1007D000CC090020710500006907000070B50B4CC2
:1007E0000B4D94F856300B4903F0FB0384F8563058
:1007F0001620A84794F85730074903F0FB0384F804
:10080000573017202B46BDE8704018470080004144
:10081000190700000200160002001700064B4022D4
:10082000C3F8E0204322C3F88C20044A936943F4C0
:1008300080639361704700BF001C004000080040C7
:1008400010B5054B054906489847064B9847BDE843
:100850001040054B184700BF1D0800000040014133
:10086000D8090020C5030000DD07000010B5044BC7
:100870009847044B9847BDE81040034B184700BF0A
:1008800019040000B107000041080000C3690B42D1
:10089000FCD170470268034B42F002020260032160
:1008A000184700BF8D0800000268034B22F00202C7
:1008B00002600321184700BF8D0800000160014B52
:1008C000032118478D08000070B50C4D06460FCD6A
:1008D00088B06C460FC495E80F0084E80F006A46A4
:1008E000002352F8041BB14202D1D8B208B070BD47
:1008F0000133082BF5D10020F8E700BFF883000092
:1009000008B5074B9847032808D000200549064B37
:1009100040F2A63298474FF0FF3008BD0020FCE7B8
:10092000C9080000DA83000079040000F8B5044625
:10093000003818BF01201049104B114E40F20562DB
:100940009847104B20469847042510274FF6FF7212
:1009500004212046B047638BC3F30113012B01D15F
:100960000020F8BD013AF3D1013D02D06783B047C2
:10097000ECE76FF00500F4E7DA830000790400008B
:100980008D080000950800004268034B42F4403295
:1009900042600421184700BF8D0800002DE9F04196
:1009A0000D4614460421534AD0F800809047438BEB
:1009B00015F0010F06469BB2174660D09D0716D56D
:1009C00001220276628892B242F48052628062888A
:1009D00003F0010522F480721204C5F1FF25120C08
:1009E00005F57F056280FC352846BDE8F08113F0EF
:1009F000040515D06368002BC1BF63889BB243F424
:100A00008053638063881F0401D53B4B98476388FC
:100A100023F480731B041B0C63806FF00105E3E774
:100A2000638813F4806713D027889047436AFF09CF
:100A300007F0060703F480433B4343F0F1034362AE
:100A40009047638823F480631B041B0C6380CBE70F
:100A5000656845B963881E0401D5274B98476388AC
:100A600023F48073F0E7D4F8088018F8013B836220
:100A7000013D9047C4F8088065600025B4E715F093
:100A80000205B1D06268002A31D059072FD4013A4B
:100A9000C8F3C06362609AB9ABB163881B0408D520
:100AA000736823F48073736004213046B847124B97
:100AB0009847638823F480731B041B0C63800BE04E
:100AC000012A09D143B1736843F480237360042180
:100AD0003046B847002AE0D004213046B847A36822
:100AE000B26A591CA1601A7002233376C5E702234B
:100AF000337692E78D080000890900002DE9F04760
:100B00000C46214BDFF88CA0204DDFF88C90064678
:100B100008469847E36913F0010FC7B213D11823B1
:100B200003FB07A303215B6A204603F01C08A847C8
:100B300023689B0703D5164B98470221A84748F026
:100B400001012046C847182202FB07A220460121C6
:100B5000A847546A2146C847936A43600421A847BE
:100B6000D36AC360C4F30163B381436AC4F34064CE
:100B700023F4804343EA84334362A847538EF381CE
:100B80000020BDE8F08700BF010900008D080000CB
:100B9000A9080000F8830000BD08000070B51A4BDA
:100BA00004469847022805D01849194B40F24722BD
:100BB00000209847E369174D174E13F0010F0DD130
:100BC000164B03212046984723689B0703D5144BF7
:100BD00098470221A84705212046B0472046012119
:100BE000A8471049B0474FF4403363601F21A8471E
:100BF0000D4BA3604DF6AD03A3810023A3731846EC
:100C000084F8303070BD00BFC9080000DA830000EE
:100C1000790400008D080000BD0800008D08000068
:100C2000A9080000040010400200700070B50546DD
:100C30000C46054B05490120BB2298472C602046F5
:100C4000034BBDE87040184779040000DA830000C8
:100C50009D0B00000068014B184700BF950800007D
:100C60000368996270470368986AC0B27047036866
:100C7000187E00F0010070470368187EC0F3400042
:100C800070470368187EC0F38000704770B5044653
:100C90000D46064B064901204FF4A3629847256193
:100CA00029462046034BBDE87040184779040000F0
:100CB000DA830000FD0A000010B50446054B064922
:100CC000012040F2355298472069044BBDE810409E
:100CD000184700BF79040000DA8300002D090000E6
:100CE0002DE9F0470446DFF85C9107690E464FF4A2
:100CF000BA6251490120C84720694F49003840F283
:100D0000D15218BF0120C847301E18BF01204A49E0
:100D100040F2D252C8476388D8057AD47388DFF886
:100D200028819BB243F48073738096E807007B6848
:100D300043F4807384E807007B6004213846C04791
:100D400025693D49D5F800A040F2A5520120C847C9
:100D50006368012B6B6839D11AF0006F36D043F409
:100D600080236B6004212846C047238859054FEA39
:100D700043022ED56388DB0741BF63889BB243F4EF
:100D8000806363800421C04722F001026B6A520530
:100D9000520D03F480431A4342F400426A62C04792
:100DA00022694FF48033117E013BC9B201D088071C
:100DB000F9D028462246214DA847D0B1638823F4B4
:100DC00080731B041B0C6380BDE8F08723F4802331
:100DD000C7E7B4F802900421C0471FFA89F96B6A8B
:100DE000D2B209F0010942EA090203F480431A432E
:100DF000D4E76388DA05E7D522694FF48033117EA2
:100E0000013BC9B208D08807F9D022463846A84726
:100E1000EFE76FF00500D7E773881B0402D5084B96
:100E200038469847638823F480731B041B0C638047
:100E30006FF00400C8E700BFDA8300009D090000DE
:100E400089090000790400008D080000004B184754
:100E50006D0800000148024B184700BFCC09002074
:100E6000B10500000FB430B5C5B0134C489D2846FD
:100E7000A047FF281CD8114B4FF48072002104A812
:100E8000984749AB4FF4807200210393009304A864
:100E90002B460B4DA84704A8A0470A4B82B204A9D1
:100EA00009489847002045B0BDE8304004B070477D
:100EB0004FF0FF30F7E700BF8119000095180000E0
:100EC000892E0000ED020000CC0900200148024BF1
:100ED000184700BFD8090020010400000A46024B51
:100EE00001460248184700BFED020000EC0900204F
:100EF0002DE9F3411848194D194EA8470024214601
:100F000030460134A847102CF9D10024154FDFF8E2
:100F10006880154E8DF80740230703D104F0F001D7
:100F20003846A8474FF4006221B24046B0470F4B05
:100F300001210DF107009847012809D00C48A84766
:100F40000134782CE8D10B48A84702B0BDE8F08105
:100F500021460348A847F3E741840000650E0000DE
:100F6000458400004B84000009040000DD0E0000F1
:100F700053840000C6830000D809002081F000419E
:100F800002E000BF83F0004330B54FEA41044FEA6E
:100F9000430594EA050F08BF90EA020F1FBF54EA09
:100FA000000C55EA020C7FEA645C7FEA655C00F0A5
:100FB000E2804FEA5454D4EB5555B8BF6D420CDD76
:100FC0002C4480EA020281EA030382EA000083EAF9
:100FD000010180EA020281EA0303362D88BF30BD99
:100FE00011F0004F4FEA01314FF4801C4CEA1131EF
:100FF00002D0404261EB410113F0004F4FEA03334E
:101000004CEA133302D0524263EB430394EA050FD8
:1010100000F0A780A4F10104D5F1200E0DDB02FA47
:101020000EFC22FA05F2801841F1000103FA0EF2DB
:10103000801843FA05F359410EE0A5F120050EF1A1
:10104000200E012A03FA0EFC28BF4CF0020C43FAD2
:1010500005F3C01851EBE37101F0004507D54FF0DF
:10106000000EDCF1000C7EEB00006EEB0101B1F52F
:10107000801F1BD3B1F5001F0CD349085FEA300075
:101080004FEA3C0C04F101044FEA445212F5800F80
:1010900080F09A80BCF1004F08BF5FEA500C50F11D
:1010A000000041EB045141EA050130BD5FEA4C0C00
:1010B000404141EB0101013C28BFB1F5801FE9D25D
:1010C00091F0000F04BF01460020B1FA81F308BF80
:1010D0002033A3F10B03B3F120020CDA0C3208DD4C
:1010E00002F1140CC2F10C0201FA0CF021FA02F127
:1010F0000CE002F11402D8BFC2F1200C01FA02F197
:1011000020FA0CFCDCBF41EA0C019040E41AA2BFBB
:1011100001EB0451294330BD6FEA04041F3C1CDA83
:101120000C340EDC04F11404C4F1200220FA04F0A3
:1011300001FA02F340EA030021FA04F345EA03014D
:1011400030BDC4F10C04C4F1200220FA02F001FA0F
:1011500004F340EA0300294630BD21FA04F0294691
:1011600030BD94F0000F83F4801306BF81F480112A
:101170000134013D4EE77FEA645C18BF7FEA655C9D
:1011800029D094EA050F08BF90EA020F05D054EA6F
:10119000000C04BF1946104630BD91EA030F1EBF74
:1011A0000021002030BD5FEA545C05D14000494178
:1011B00028BF41F0004130BD14F580043CBF01F56B
:1011C000801130BD01F0004545F0FE4141F4700151
:1011D0004FF0000030BD7FEA645C1ABF194610462C
:1011E0007FEA655C1CBF0B46024650EA013406BF2D
:1011F00052EA033591EA030F41F4002130BD00BFEC
:1012000090F0000F04BF0021704730B54FF48064A8
:1012100004F132044FF000054FF0000150E700BF29
:1012200090F0000F04BF0021704730B54FF4806488
:1012300004F1320410F0004548BF40424FF0000175
:101240003EE700BF42004FEAE2014FEA31014FEAB8
:1012500002701FBF12F07F4393F07F4F81F0605107
:10126000704732F07F4208BF704793F07F4F04BF52
:1012700041F40021704730B54FF4607401F000452F
:1012800021F000411CE700BF50EA010208BF70478F
:1012900030B54FF000050AE050EA010208BF704780
:1012A00030B511F0004502D5404261EB41014FF4E9
:1012B000806404F132045FEA915C3FF4D8AE4FF0F1
:1012C00003025FEADC0C18BF03325FEADC0C18BFD4
:1012D000033202EBDC02C2F1200300FA03FC20FA25
:1012E00002F001FA03FE40EA0E0021FA02F1144472
:1012F000BDE600BF70B54FF0FF0C4CF4E06C1CEA8B
:1013000011541DBF1CEA135594EA0C0F95EA0C0FFB
:1013100000F0DEF82C4481EA030621EA4C5123EA6E
:101320004C5350EA013518BF52EA033541F480119D
:1013300043F4801338D0A0FB02CE4FF00005E1FB50
:1013400002E506F00042E0FB03E54FF00006E1FB9A
:1013500003569CF0000F18BF4EF0010EA4F1FF04DD
:10136000B6F5007F64F5407404D25FEA4E0E6D411D
:1013700046EB060642EAC62141EA55514FEAC5202E
:1013800040EA5E504FEACE2EB4F1FD0C88BFBCF5AA
:10139000E06F1ED8BEF1004F08BF5FEA500E50F15B
:1013A000000041EB045170BD06F0004646EA010121
:1013B00040EA020081EA0301B4EB5C04C2BFD4EB53
:1013C0000C0541EA045170BD41F480114FF0000E4C
:1013D000013C00F3AB8014F1360FDEBF002001F0BA
:1013E000004170BDC4F10004203C35DA0C341BDC34
:1013F00004F11404C4F1200500FA05F320FA04F006
:1014000001FA05F240EA020001F0004221F0004139
:1014100010EBD37021FA04F642EB06015EEA430EAC
:1014200008BF20EAD37070BDC4F10C04C4F12005DC
:1014300000FA04F320FA05F001FA04F240EA02008F
:1014400001F0004110EBD37041F100015EEA430E60
:1014500008BF20EAD37070BDC4F1200500FA05F280
:101460004EEA020E20FA04F301FA05F243EA0203FF
:1014700021FA04F001F0004121FA04F220EA02000E
:1014800000EBD3705EEA430E08BF20EAD37070BD54
:1014900094F0000F0FD101F00046400041EB010134
:1014A00011F4801F08BF013CF7D041EA060195F016
:1014B000000F18BF704703F00046520043EB0303D0
:1014C00013F4801F08BF013DF7D043EA06037047BD
:1014D00094EA0C0F0CEA135518BF95EA0C0F0CD0C8
:1014E00050EA410618BF52EA4306D1D181EA03010E
:1014F00001F000414FF0000070BD50EA410606BF08
:101500001046194652EA430619D094EA0C0F02D14C
:1015100050EA013613D195EA0C0F05D152EA033691
:101520001CBF104619460AD181EA030101F00041AF
:1015300041F0FE4141F470014FF0000070BD41F0F8
:10154000FE4141F4780170BD70B54FF0FF0C4CF4D2
:10155000E06C1CEA11541DBF1CEA135594EA0C0FF1
:1015600095EA0C0F00F0A7F8A4EB050481EA030E3E
:1015700052EA03354FEA013100F088804FEA033325
:101580004FF0805545EA131343EA12634FEA0222F3
:1015900045EA111545EA10654FEA00260EF00041B4
:1015A0009D4208BF964244F1FD0404F5407402D206
:1015B0005B084FEA3202B61A65EB03055B084FEA97
:1015C00032024FF480104FF4002CB6EB020E75EB94
:1015D000030E22BFB61A754640EA0C005B084FEABC
:1015E0003202B6EB020E75EB030E22BFB61A754639
:1015F00040EA5C005B084FEA3202B6EB020E75EB84
:10160000030E22BFB61A754640EA9C005B084FEAFB
:101610003202B6EB020E75EB030E22BFB61A754608
:1016200040EADC0055EA060E18D04FEA051545EAF7
:1016300016754FEA06164FEAC30343EA52734FEAA0
:10164000C2025FEA1C1CC0D111F4801F0BD141EA19
:1016500000014FF000004FF0004CB6E711F4801F7E
:1016600004BF01430020B4F1FD0C88BFBCF5E06F5E
:101670003FF6AFAEB5EB030C04BFB6EB020C5FEA6E
:10168000500C50F1000041EB045170BD0EF0004EC3
:101690004EEA113114EB5C04C2BFD4EB0C0541EAF5
:1016A000045170BD41F480114FF0000E013C90E6F2
:1016B00045EA060E8DE60CEA135594EA0C0F08BFB6
:1016C00095EA0C0F3FF43BAF94EA0C0F0AD150EAB5
:1016D00001347FF434AF95EA0C0F7FF425AF104648
:1016E00019462CE795EA0C0F06D152EA03353FF470
:1016F000FDAE1046194622E750EA410618BF52EAED
:1017000043067FF4C5AE50EA41047FF40DAF52EAC0
:1017100043057FF4EBAE12E770B50D4E0D4D761B11
:10172000B61006D0002455F8043B01349847A64271
:10173000F9D1094E094D761B07F0A6F8B61006D070
:10174000002455F8043B01349847A642F9D170BDF6
:101750009488000094880000988800009488000015
:10176000844641EA000313F003036DD1403A41D3AC
:1017700051F8043B40F8043B51F8043B40F8043B6B
:1017800051F8043B40F8043B51F8043B40F8043B5B
:1017900051F8043B40F8043B51F8043B40F8043B4B
:1017A00051F8043B40F8043B51F8043B40F8043B3B
:1017B00051F8043B40F8043B51F8043B40F8043B2B
:1017C00051F8043B40F8043B51F8043B40F8043B1B
:1017D00051F8043B40F8043B51F8043B40F8043B0B
:1017E00051F8043B40F8043B51F8043B40F8043BFB
:1017F000403ABDD2303211D351F8043B40F8043B9B
:1018000051F8043B40F8043B51F8043B40F8043BDA
:1018100051F8043B40F8043B103AEDD20C3205D3AA
:1018200051F8043B40F8043B043AF9D2043208D0A2
:10183000D2071CBF11F8013B00F8013B01D30B8814
:1018400003806046704700BF082A13D38B078DD0F2
:1018500010F003038AD0C3F10403D21ADB071CBFC4
:1018600011F8013B00F8013B80D331F8023B20F82E
:10187000023B7BE7043AD9D3013A11F8013B00F867
:10188000013BF9D20B7803704B7843708B788370EF
:1018900060467047830730B548D0541E002A3FD0B9
:1018A000CAB2034601E0013C3AD303F8012B9D077D
:1018B000F9D1032C2DD9CDB245EA05250F2C45EAE7
:1018C000054536D9A4F1100222F00F0C03F1200EC9
:1018D000E6444FEA121C03F1100242E9045542E9C2
:1018E000025510327245F8D10CF1010214F00C0FC0
:1018F00003EB021204F00F0C13D0ACF1040323F03D
:1019000003030433134442F8045B9342FBD10CF00D
:1019100003042CB1C9B21C4403F8011B9C42FBD147
:1019200030BD64461346002CF4D1F9E70346144653
:10193000BFE71A46A446E0E70FB400B5074983B0F5
:1019400004AB086853F8042B8168019300F086F813
:1019500003B05DF804EB04B0704700BF0000002046
:101960000000000000000000000000000000000077
:101970000000000000000000000000000000000067
:1019800090F800F06DE9024520F007016FF0000CBF
:1019900010F0070491F820F040F049804FF0000467
:1019A0006FF00700D1E9002391F840F000F1080042
:1019B00082FA4CF2A4FA8CF283FA4CF3A2FA8CF37A
:1019C0004BBBD1E9022382FA4CF200F10800A4FAE1
:1019D0008CF283FA4CF3A2FA8CF3E3B9D1E9042335
:1019E00082FA4CF200F10800A4FA8CF283FA4CF36C
:1019F000A2FA8CF37BB9D1E9062301F1200182FA26
:101A00004CF200F10800A4FA8CF283FA4CF3A2FA2B
:101A10008CF3002BC6D0002A04BF04301A4612BA39
:101A2000B2FA82F2FDE8024500EBD2007047D1E93C
:101A3000002304F00305C4F100004FEAC50514F0CB
:101A4000040F91F840F00CFA05F562EA05021CBF9C
:101A500063EA050362464FF00004A9E72DE9F04F61
:101A6000BFB01C468A46904605460C9002F024FD05
:101A70000268159210460D94FFF782FF13901DB176
:101A8000AB6B002B00F0D781BAF90C3099049AB2F5
:101A90000AD443F40053AAF80C309AB2DAF8603052
:101AA00023F40053CAF86030170740F1AC80DAF82D
:101AB0001030002B00F0A78002F01A020A2A00F072
:101AC000B0800023CDE92233129314931693099327
:101AD00000240023CDE910342EAA21929146D3464A
:101AE00098F80030002B00F05381444604E014F8CD
:101AF000013F002B00F0A380252BF8D1B4EB0805A3
:101B000040F0A1802378002B00F042810023621C6A
:101B10008DF8673018464FF0FF3519461C46904641
:101B200018F8017BA7F12002582A00F2A780DFE80D
:101B300012F0EF01A500A500EC01A500A500A5008D
:101B4000A500A500A500B8018406A500C001C30139
:101B5000A500E901590059005900590059005900E0
:101B6000590059005900A500A500A500A500A50031
:101B7000A500A500A500A500A500DD013D01A5006B
:101B80003D01A500A500A500A5003802A500A500FF
:101B90004502A500A500A500A500A5003B02A500E3
:101BA000A5000402A500A500A500A500A500A500AC
:101BB000A500A500A500A500F50186013D013D0198
:101BC0003D01DA018601A500A5006700A500BA0263
:101BD000A7028C026700A5006602A5005702A500B7
:101BE000A5004F02A7F13002002118F8017B01EB9C
:101BF000810102EB4101A7F13002092AF5D991E7F1
:101C000044F010048CE70C98514601F053F9002879
:101C100041F09680BAF80C2002F01A020A2A7FF4EA
:101C200050AFBAF90E30002BFFF64BAF0C9823469D
:101C3000424651463FB0BDE8F04F01F0EFB8B4EB7B
:101C4000080500F0A580239B2B442393229B01339E
:101C5000072BC9E90085229305DC09F10809099BD6
:101C60002B4409934EE70C9821AA594603F030FC07
:101C7000002840F04A830DF1B809F0E70B91002BE2
:101C800040F08B87002F00F0838000238DF86730B1
:101C900001238DF8907007930A9324AD00230694D6
:101CA00008930F93069B13F0020302D0079A0232A7
:101CB0000792069A239C12F084020E9205D10B9A89
:101CC0000799561A002E00F383839DF867208AB186
:101CD000229A0DF1670101320134C9F80010072A78
:101CE0004FF0010123942292C9F8041000F3C48339
:101CF00009F1080983B1229B1AAA01330234C9F8F9
:101D00000020072B4FF0020223942293C9F80420ED
:101D100000F3A68309F108090E9B802B00F0618275
:101D2000089B0A9AA3EB020ABAF1000F00F3A38200
:101D3000069BDB0500F1E9810A9BC9F804301C44CD
:101D4000229BC9F800500133072B2394229300F300
:101D5000E98209F10809069B590705D50B9B079AEB
:101D60009D1A002D00F39683099B0B9A07998A42CE
:101D7000ACBF9B185B180993002C40F0BE82002377
:101D8000229398F800300DF1B809002B7FF4ADAE26
:101D9000239BDA46002B40F0F986BAF80C305A063D
:101DA00000F1CE8709983FB0BDE8F08F0B91089500
:101DB000002B40F0A8870D9B073323F00701F1E8C3
:101DC000022323F00045CDE910230D91164610465D
:101DD000A64B29464FF0FF3206F06AFA002840F081
:101DE0007D84A24B304629464FF0FF3206F042FA7E
:101DF000002840F07384DDE910010022002306F082
:101E00002FFA002840F0A9869DF86710984D24F01D
:101E100080030693974B0022472FC8BF1D4603231C
:101E2000CDE907320A930F9200293FF43BAF079B9D
:101E30000133079336E70C9802F0C8F924E60B91BA
:101E40000895002B40F053870D9BE50653F8042BB3
:101E50000D9302D4600600F138841346002AC0F2C4
:101E6000258408989DF86710013006D024F0800082
:101E70000690002A00F0D883069C092B00F24585C5
:101E800030338DF8B730012306940A930DF1B7056E
:101E9000089B0A9A9342B8BF1346079300230F93F7
:101EA000C2E70D9A52F8041B002980F208844942C7
:101EB0000D9244F0040433E618F8017B2A2F00F059
:101EC0009B87A7F13002092A4FF000053FF62AAEA2
:101ED00018F8017B05EB850502EB4505A7F13002FB
:101EE000092AF5D91EE644F0400419E60B9108953D
:101EF000002B40F0F0860D9B53F8042B0D9344F01B
:101F00001004AAE744F080040AE644F0010407E65E
:101F100000287FF405AE0123202001E60D9B0B91E4
:101F200000228DF8672053F8042B0D9301238DF8C0
:101F3000902007930A9324ADB0E60B910895002BEF
:101F400040F0E5864C4B14930D9AE10652F8043BA1
:101F50000D9202D4620648BF9BB2E60702D5002B61
:101F600040F061840222002108988DF86710451C1A
:101F700000F0AF8024F080050695002B40F0A8808B
:101F8000002840F01A81002A40F0528314F0010327
:101F90000A9300F0978330238DF8B7300DF1B70521
:101FA00076E744F00804BBE50D9A0B9152F8043B28
:101FB000089544F010040D920122D4E70D9A0B917C
:101FC00052F8043B089544F010040D920022CAE731
:101FD0000B910895002B40F08286284B1493B3E7B1
:101FE0000B910895002B40F07E860D9AE60652F87C
:101FF000043B0D92E0D4600648BF9BB2DCE70D9E27
:10200000089556F8045B089B0B914FF0000A8DF879
:1020100067A0002D00F02E845A1C00F02E851A4671
:102020005146284602F06CFD002800F04986431B0B
:102030000A9323EAE3739DF86710CDF820A00D966C
:1020400006940793CDF83CA0EEE60D9A0B9152F85A
:10205000043B0D9247F63002ADF86820074A14920F
:10206000089544F00204022278277CE7FFFFEF7F07
:10207000588400005C840000688400007C840000B8
:102080000B910895002B40F036860D9A14F0100144
:1020900052F8043B0D9299D114F040023FF463AF23
:1020A0009BB20A465FE7002B40F029860D9AE006B6
:1020B00002F1040307D461060D9A04D51268099948
:1020C00011800D930CE51268099911600D9307E5D5
:1020D000069C012A3FF4D1AE022A74D02EAD03F043
:1020E00007023032DB08284605F8012DF7D1E60754
:1020F00072D5302A70D03023023805F8013C2EAB5F
:102100001B1A06940A930546C2E6652F40F3158113
:10211000DDE910010022002306F098F8002800F005
:10212000F481229BB14AC9F8002001330134012215
:10213000072B23942293C9F8042000F3428409F169
:1021400008091B9B129A934280F2B482139B159A42
:102150001C44C9E90023229B23940133072B2293BB
:1021600000F37C8309F10809129B5D1E002D7FF7A7
:10217000F2AD102D229B9E4E40F3C980DDF830A0B9
:10218000102705E009F10809103D102D40F3BF802C
:1021900001331034072BC9E90067CDE92234F1DDA2
:1021A00021AA5946504603F093F9002840F0AD802B
:1021B000DDE922340DF1B809E6E7012A00F01E85B9
:1021C000022A069C8AD114982EAD03F00F021B0937
:1021D000825C05F8012DF8D12EAB5B1B06940A93A7
:1021E00056E60B9B079AA3EB020ABAF1000F7FF7A2
:1021F00097ADBAF1100F229B7D4E2EDD32460E9523
:102200005E460C9DBB46174606E0AAF1100ABAF1DD
:10221000100F09F108091BDD013310341022072BC0
:10222000CDE92234C9F80070C9F80420EDDD21AAF7
:10223000314628460DF1B80903F04AF9002840F06C
:102240006281AAF1100ABAF1100FDDE92234E3DC51
:102250003A460E9D5F46B346164601335444072B5B
:10226000CDE92234C9F80060C9F804A000F3B683B0
:1022700009F1080954E5BAF1100F229B5C4E2EDDDE
:10228000324608955E460C9DBB46174606E0AAF10D
:10229000100ABAF1100F09F108091BDD01331034DF
:1022A0001022072BCDE92234C9F80070C9F80420A8
:1022B000EDDD21AA3146284603F00AF9002840F056
:1022C0002281AAF1100ABAF1100FDDE922340DF1D2
:1022D000B809E3DC3A46089D5F46B346164601332B
:1022E0005444072BCDE92234C9F80060C9F804A092
:1022F00000F3CF8109F108091AE50C9821AA594683
:1023000003F0E6F800283FF43AADDA4645E501333C
:102310002C44072BC9F80060C9F80450CDE92234D9
:102320007FF717AD0C9821AA594603F0D1F8002881
:10233000EBD1239C0DF1B8090DE5129B229F012BD7
:1023400004F1010407F1010709F1080A40F3518182
:102350000123072FCDE92274C9F80050C9F80430D1
:1023600000F3B982139B159A01371C44072FCAE961
:102370000023CDE9227400F3BB820AF1080A129B04
:10238000DDE9100103F1FF390022002305F05EFFB3
:10239000002840F05281013701354C44072FCDE928
:1023A0002274CAF80050CAF8049000F330810AF190
:1023B000080A169BCAF8043001371C44072F1DABCE
:1023C000CDE92274CAF80030ACDC0AF10809C2E495
:1023D000102E229A35DD59461793B34623462E46D2
:1023E0000C9C4FF0100A0D460BE000BF98840000D3
:1023F000AC840000ABF1100BBBF1100F09F1080920
:1024000019DD0132B3491033072AC9E9001ACDE9B1
:102410002223EFDD21AA294620460DF1B80903F059
:1024200057F8002840F0CA82ABF1100BBBF1100F37
:10243000DDE92223E5DC29461C46179B35465E462E
:102440008B460132A349C9F804603444072ACDE918
:102450002224C9F8001000F3A28209F1080934E42B
:102460000C9821AA594603F033F800287FF44DAFA9
:10247000239C0DF1B8094FE40C98179321AA5946F3
:1024800003F026F800287FF440AF239C179B0DF142
:10249000B8092FE4102D229B1FDD0C9F102604E0AD
:1024A000103D102D09F1080917DD0133894A103458
:1024B000072BC9E90026CDE92234F1DD21AA5946CE
:1024C00038460DF1B80903F003F800287FF41DAF7A
:1024D000103D102DDDE92234E7DC01337D4AC9F8D7
:1024E00004502C44072BCDE92234C9F800207FF793
:1024F0003BAC0C9821AA594602F0EAFF00287FF471
:1025000004AF239C30E4B24647E41B99002940F312
:1025100012820F9E129B9E42A8BF1E46002E0BDD0C
:10252000229B01333444072BC9E90056239422939C
:1025300000F3A88309F108090F9F002EA8BFBF1B55
:10254000002F00F3A0811B9A129B9A4280F279819E
:10255000139B15991C44C9E90013229B2394013352
:10256000072B229300F3738309F10809129B0F993B
:102570009A1A5E1A9642A8BF1646002E0EDD229BBE
:10258000C9F8046001330D443444072BC9F80050E6
:102590002394229300F3858309F10809002EACBF30
:1025A000951B1546002D7FF7D6AB102D229B4A4E6A
:1025B0007FF7ADAEDDF830A0102705E009F108097E
:1025C000103D102D7FF7A3AE01331034072BC9E95E
:1025D0000067CDE92234F1DD21AA5946504602F0C8
:1025E00077FF00287FF491AEDDE922340DF1B809C0
:1025F000E6E7069BD8073FF5ABAE0123072FCDE9F1
:102600002274C9F80050C9F804307FF7D2AE0C9894
:1026100021AA594602F05CFF00287FF476AEDDE97E
:1026200022740DF1B80AC4E6089A002A40F0E68246
:10263000002308930A932EAD2AE4B9F1000F7FF727
:10264000B8AEB9F1100F244E40F30B82CDF82080C4
:102650001025DDF8308007E00AF1080AA9F1100919
:10266000B9F1100F40F3FB8101371034072FCAE98D
:102670000065CDE92274EFDD21AA5946404602F0FB
:1026800027FF00287FF441AEDDE922740DF1B80A7E
:10269000E4E70C9821AA594602F01AFF00287FF4BB
:1026A00034AE239C0DF1B809FFF742BB53422D21F4
:1026B000012259E4069BDF077FF54DAB46E50D92FD
:1026C000FFF72EBA2EADFFF7E3BB12B21346FFF7AA
:1026D000C5BB00BF9C840000AC840000DDE9100194
:1026E00002460B4605F0E4FD002840F04F83089AAF
:1026F00027F02003511C0A9300F0D082472B00F0F2
:102700005D82DDE9101244F4807306931346002BBA
:10271000C0F228820793DDF840A000230E93662FB5
:1027200000F0C681462F00F0C3810A9B452B52461C
:10273000079B00F066821FA904911CA903911BA9A5
:10274000089E029102210C980196009100F0D0FCA5
:10275000672F054640F05B83E30700F164821F9B0F
:102760005B1B12931B9B0F930A9B472B07D10F9B5D
:10277000DE1C03DB089A9A4280F27682023F0F9AAF
:102780008DF87470531E002B1B93B6BFC2F101036A
:102790002B222D22092B8DF8752040F3BC820DF1E0
:1027A0008306DFF8F8C2324610468CFB0321DA17A5
:1027B000C2EBA10202EB8201A3EB4101303100F830
:1027C000011C19466329134600F1FF32ECDC30335B
:1027D000D9B2831E9E4202F8011C40F215831346B3
:1027E0000DF1760201E013F8011B02F8011B9E4275
:1027F000F9D10DF185030DF176021B1A13441DAAC0
:102800009B1A1693129A169B012A13440A9340F3BB
:10281000B4820A9B139A13440A9323EAE37307933F
:1028200000230F937DE130228DF868208DF86970C8
:1028300044F002040222FFF796BB01232B20FFF78E
:102840006FB9069BDE073FF583AE129B0F999A1A6C
:102850005B1A9342A8BF13461E469FE60C9821AA16
:10286000594602F035FE00287FF44FAD239C0DF150
:10287000B80979E4062B28BF0623894D0A930D96E3
:102880000793FFF70BBA102F229B864E40F3588117
:10289000324608955E460C9D4FF0100A934605E0BF
:1028A00009F10809103F102F40F34681013310341D
:1028B000072BC9E900BACDE92234F1DD21AA31465E
:1028C000284602F005FE00287FF41DAEDDE9223423
:1028D0000DF1B809E6E70C9821AA594602F0F8FD77
:1028E00000287FF412ADDDE922740DF1B80A39E554
:1028F0000C9821AA594602F0EBFD00287FF405ADA3
:10290000DDE922740DF1B80A39E5674E2EADA6FB5C
:102910000302D20802EB8200A3EB4000303005F83E
:10292000010D184609281346F1D82EAB5B1B0694FF
:102930000A93FFF7ADBA229B5C4AC9F80020013325
:1029400001340122072B23942293C9F8042000F3B9
:10295000108109F1080900294DD1069B129A03F054
:10296000010313433FF4F7A9139B15991A19C9E9F9
:102970000013229B23920133072B229300F324811F
:1029800009F108091299C9F8005001338C18072B76
:10299000CDE92234C9F804107FF7DBA9C2E40C9812
:1029A000179321AA594602F093FD00287FF4ADAC9D
:1029B000239C179B0DF1B809FFF787B9AA46FFF7CB
:1029C000ECB90C9821AA594602F082FD00287FF448
:1029D0009CAC239C0DF1B809FFF7B3BB0C9821AA5E
:1029E000594602F075FD00287FF48FAC239C0DF151
:1029F000B809FFF795B9139B15981A19C9E900038F
:102A0000229B23920133072B229300F3DD8009F1EF
:102A100008090029B6DA4F421031224E80F2958122
:102A2000DDF830A0102405E009F10809103F102F4F
:102A300040F38B8101331032072BC9E90064CDE9E3
:102A40002232F1DD21AA5946504602F041FD00280C
:102A50007FF45BACDDE922320DF1B809E6E7DDF881
:102A60002080CAF8006001374C44072FCDE922745A
:102A7000CAF804907FF79BACC9E52846CDF820A0A2
:102A80000D960694FEF77CFF20EAE0739DF8671030
:102A90000A900793CDF83CA0FFF7C6B96766666653
:102AA00090840000AC840000CDCCCCCC9884000095
:102AB0001FA9DDE9073604911CA903911BA9029106
:102AC000032101960C980091524600F011FB054637
:102AD00086192B78302B64D01B9B1E4407995046D7
:102AE0000022002305F0B2FB002800F09E80334650
:102AF0005B1B12931B9B0F930A9B472B3FF437AE34
:102B0000662F7FF43CAE089A04F0010313430F9A3A
:102B1000002A40F36981002B40F049810F9B079305
:102B20000A930E9B002B00F08C802D238DF86730CC
:102B300000230893FFF77BB95A46089DB346164613
:102B400001333C44072BCDE92234C9F80060C9F8B1
:102B5000047047DC09F10809F5E42D218DF86710B0
:102B6000FFF754B903F1004307932D238A460E93D0
:102B7000D5E50C9821AA594602F0AAFC00287FF45A
:102B8000C4AB1B99239C0DF1B809E4E60C9821AA6B
:102B9000594602F09DFCFFF700B98DF86700FFF77A
:102BA00071B8079950460022002305F04FFB00281A
:102BB00092D1089BC3F101031B938EE7002A1346B1
:102BC00008BF012308939CE50C9821AA594602F0FE
:102BD0007FFC00287FF499ABDDE922321B990DF1CF
:102BE000B80916E70C9821AA594602F071FC002892
:102BF0007FF48BAB239C0DF1B809A4E4069CFFF78E
:102C00003FB908990C984E1C1FA904911CA9039167
:102C10001BA9029102210196009100F069FA054674
:102C2000472F3FF499AD2E4458E71F9BB342BFF4A2
:102C30005FAF30215A1C1F9219701F9B9E42F9D81A
:102C400056E70E9B9DF867100893FFF7EDB80C98B8
:102C500021AA594602F03CFC00287FF456AB1B9A8F
:102C6000239C0DF1B80981E4129B0F9A93425BDC1F
:102C7000E4070F9B00F1A58023EAE37207920A9311
:102C800067274EE70C9821AA594602F021FC00283C
:102C90007FF43BAB239C0DF1B8094DE40623089368
:102CA0002FE50C9821AA594602F012FC00287FF467
:102CB0002CAB1B9A129B239C9A1A0DF1B8096DE458
:102CC000089B9DF867100D96069407930A93089049
:102CD0000F90FFF7A9B88DF86700FFF70CB98DF8D2
:102CE0006700FFF77AB98DF86700FFF77EB98DF8B6
:102CF0006700FFF7A9B88DF86700FFF7C6B98DF830
:102D00006700FFF7D3B98DF86700FFF754B88DF867
:102D10006700FFF717B930338DF8773030238DF81F
:102D20007630042316936DE5DDE9123213440F9AD1
:102D30000A93002A4DDD23EAE37307936727F0E641
:102D40004FF0FF330993FFF72DB801333A44072BB7
:102D5000CDE92232C9F80060C9F804707FF710AEDF
:102D60000C9821AA594602F0B3FB00287FF4CDAAA3
:102D7000DDE922320DF1B80904E614F001020F92E8
:102D80007FF447AD23EAE3730793CAE6119B214D15
:102D9000002BB8BF2D2124F080030693A8BF9DF817
:102DA00067101D4BB8BF8DF86710FFF734B80F9B45
:102DB000139A1344089A1A4422EAE2730A92079378
:102DC000AFE6139A13440A9323EAE3730793672742
:102DD000A7E60F9B0A9AC3F101031A4422EAE273A1
:102DE0000A92079367279CE61BB9012307930A936E
:102DF00097E6139B0133DDE70D9A52F8045B0D92C1
:102E000045EAE575FEF78CBE02231693FAE4089EA8
:102E100006E700BF608400006484000070B50C46C3
:102E20008989ADF58D6D21F00201ADF81010216E8C
:102E30001991E189ADF81210E1690891616A0A916E
:102E40001AA9019105914FF4806103910691002127
:102E5000079101A90646FEF701FE051E07DB01A941
:102E6000304601F02BF9002818BF4FF0FF35BDF8B0
:102E700010305B0603D5A38943F04003A3812846A5
:102E80000DF58D6D70BD00BF10B5141E1946029B67
:102E900008DB0A46214603F0C5F8002801DBA04202
:102EA00005D210BDBDE810401A4603F0F3B800F09B
:102EB0006BF800BF38B5334B1B6805460C460BB1A9
:102EC0009A6B12B3B4F90C3018079AB225D5216960
:102ED00000292DD012F0010007D00020A060606909
:102EE0004042A06139B1002038BD950758BF6069E4
:102EF000A0600029F7D1120658BF0846F4D543F068
:102F00004003A3814FF0FF3038BD184601F05EF951
:102F1000B4F90C3018079AB2D9D4D1062AD5520781
:102F200014D4216943F00803A3819AB20029D1D1B6
:102F300002F42070B0F5007FCCD02146284601F085
:102F4000BFFAB4F90C3021699AB2C3E7216B51B1D1
:102F500004F14002914204D0284601F08DF9B4F901
:102F60000C300022226321690022C4E9001223F000
:102F70002403D7E7092243F040032A604FF0FF30D3
:102F8000A38138BD0000002000B50E4C0FCC8DB0E1
:102F9000EC46ACE80F000FCCACE80F0094E80F0053
:102FA000ACE807006846ACF80030FEF7E9FC69467B
:102FB0000246022002F044FA062002F0B5F97F2012
:102FC000FDF7C6F9BC8400002DE9F04F03690C69D8
:102FD000A34283B0C0F28880013C01F11405A30034
:102FE00000F11408009355F8243058F824200133D8
:102FF0008A469A4208EB8401814605EB84070191D9
:10300000B2FBF3F63AD34FF0000CAE4640466246B0
:1030100063465EF804BB01681FFA8BFC06FB0C33A9
:103020004FEA134C4FEA1B4B06FB0BCC9BB2D31A57
:103030001FFA8CF213FA81F3C2EB114202EB234226
:103040009BB243EA0243774540F8043B4FEA2242F1
:103050004FEA1C43DDD2009B58F8033073B9019B43
:10306000043B984504D307E0984504F1FF3403D2AC
:1030700053F80429002AF7D0C9F8104051464846B1
:1030800002F016F800282BDB01364146002355F8E4
:10309000040BD1F800C082B29A1A030C12FA8CF217
:1030A000C3EB1C4303EB224392B242EA0342AF421A
:1030B00041F8042B4FEA2343E9D258F8242008EBC7
:1030C00084036AB9043B984504D307E0984504F1AA
:1030D000FF3403D253F80429002AF7D0C9F810406E
:1030E000304603B0BDE8F08F002003B0BDE8F08F9C
:1030F0002DE9F04F016C9FB016461F46CDE90467DD
:103100002B9C824649B1426C4A60012393408B60FC
:1031100001F070FD0023CAF84030B7F10008B4BFD9
:10312000012300232360764BBCBF28F00048CDF874
:10313000148033EA080300F0AC80DDE90434002297
:10314000184621460023CDE90A0105F07FF805461F
:1031500078B12A9A012313602C9B002B00F09183F5
:10316000684B2C9A1360013B039303981FB0BDE892
:10317000F08F1CAB01931DAB00935046DDE90A2391
:1031800002F060F85FEA1854834640F09880DDE969
:103190001C542C4404F23243202B40F38883C3F1A7
:1031A000400308FA03F804F2124326FA03F348EA4C
:1031B0000300FEF725F80123013CA1F1F8711293F9
:1031C000514B0022FDF7DEFE47A3D3E90023FEF7B3
:1031D00091F847A3D3E90023FDF7D6FE0646204623
:1031E0000F46FEF71DF844A3D3E90023FEF782F84B
:1031F00002460B4630463946FDF7C6FE06460F46E8
:1032000005F06CF8002280460690002330463946CF
:1032100005F026F8002840F026832D1B069C6B1E27
:10322000162C089300F21383384B03EBC403D3E945
:103230000023DDE90A0105F013F800286CD0631EB5
:10324000069300230F936B1E002BC0F2068300230E
:103250000C93069B002B65DA069B0C9A0D93D21AF1
:10326000C3F1000900230693289B0C92092B63D815
:10327000052B40F31A83043B28930024289B023B30
:10328000032B00F25A86DFE813F01E041B0412041D
:10329000F3032A9AC8F3130842F20F7358EA060898
:1032A00013601AD12C9B002B00F05786184B039308
:1032B00008332C9A039813601FB0BDE8F08FDDE946
:1032C0000A12C2F31303084643F07F511295A4F289
:1032D000FF341C9D41F4401172E72C9B002B40F001
:1032E000B5830C4B039340E761436F63A787D23FDD
:1032F000B3C8608B288AC63FFB799F501344D33FE5
:103300000000F07F998400000000F83F2086000054
:10331000EC840000F88400006B1E002BC0F27A845D
:103320000F900C90089B069A0D9213440893289BCB
:10333000092B4FF000099BD90023CDE92833012444
:103340004FF0FF330E940993099B13930021CAF8A1
:103350004410504601F028FC0390002800F0F68548
:10336000039BCAF84030099B0E2B00F2F980002C19
:1033700000F0F6800D99002940F34E84BB4B01F01C
:103380000F0203EBC203C805D3E900454FEA21163B
:1033900040F1DC83B64BDDE90A01D3E90823FEF7EF
:1033A000D3F8CDE9100106F00F064FF0030886B1FF
:1033B000AF4FF10709D520462946D7E90023FDF78D
:1033C00099FF08F1010804460D46761007F1080739
:1033D000EFD1DDE9100122462B46FEF7B5F806468F
:1033E0000F460F9B43B1A34B00223046394604F0F1
:1033F00037FF002840F01D854046FDF711FF32469B
:103400003B46FDF777FF9C4B0022FDF7BDFDA1F188
:103410005073CDE914011593099B002B00F0DB8359
:103420000D9B1A93099B1093DDE9143403993046E0
:1034300001F101083946CDE9163404F04FFF00F1DF
:103440003003DCB2109D894B149403EBC50353E9A0
:103450000212CDE91812FDF7E3FE0B46024639468B
:103460003046FDF78FFD0E9B04460D46002B00F005
:103470008B84DDE9182381490020FEF765F8DDE93A
:103480001623FDF77FFD039F149E3E7002460B46F8
:10349000CDE9142322462B4604F000FF002840F01B
:1034A000C0840027CDF86C90CDF858B0CDF860A05E
:1034B000B946DDE914AB2BE0109B09F101099945F0
:1034C00048DA6F4B504659460022FDF713FF6C4B0C
:1034D000002282468B4620462946FDF70BFF0F4609
:1034E000064604F0FBFE0546FDF79AFE02460B4633
:1034F00030463946FDF746FD303508F8015B524647
:103500005B4604460D4604F0ABFE002840F0E9841B
:1035100022462B4657490020FDF734FD52465B46B4
:1035200004F09EFE0028C7D01A9CDDF858B0DDF8E4
:1035300060A0039A4646013402E0B24200F0A6843D
:10354000B04616F8013D392BF7D00133DBB23370AA
:10355000049468E1DDF86C90DDF858B0DDF860A007
:103560001D9B002BC0F290800D9A0E2A00F38C80D8
:103570003E4B03EBC203D3E90089299B002B1BDAE6
:10358000099B002B18DC40F041833E4B494600224A
:103590004046FDF7AFFE02460B46DDE90A0104F0A6
:1035A00069FEDDF824904C46002800F0A382299B98
:1035B000DDF80C80DF43A4E2DDE90A4542464B46D4
:1035C00020462946FDF7C0FF04F088FE0746FDF7B8
:1035D00027FE42464B46FDF78DFE039E0B460246F4
:1035E00029462046FDF7CEFC07F1300306F8013BE3
:1035F000099B012B00F07D83CDF818A00127CDF8A1
:1036000010B09A461CE042464B4620462946FDF73C
:103610009BFF04F063FE8346FDF702FE42464B46E5
:10362000FDF768FE01370B46024629462046FDF7A6
:10363000A9FC0BF13003574506F8013B00F0548319
:103640000F4B0022FDF756FE0022002304460D46D4
:1036500004F0FCFD0028D6D00D9BDDF810B0DDF89D
:1036600018A001330493B046DDE000BF20860000BF
:10367000F88500000000F03F00001C400000E03F23
:1036800000002440000014400E9A002A00F0FF8041
:10369000289A012A40F37982099B5E1EB14580F287
:1036A0004182069AA6EB09031A44B1460692002607
:1036B000099B002BC0F25283089A1A4408920C9A74
:1036C00015461A440C920121504601F03DFB044678
:1036D00065B1089900290B4608DD0C9AA942A8BFDC
:1036E0002B46D21AED1ACB1A0C920893B9F1000F9F
:1036F0000AD00E9B002B00F0D382002E00F315821F
:10370000B9EB060240F03A830121504601F01CFB60
:10371000069A002A814600F3CF80289B012B40F3B4
:103720009B810027069B0120002B40F0CF80089B47
:10373000184410F01F0000F08D81C0F12003042B0D
:1037400000F3A98040F009820C9B002B05DD59464F
:103750001A46504601F034FC8346089B002B05DDD9
:1037600049461A46504601F02BFC81460F9B002B20
:1037700040F05081099B002B40F337810E9B002BBA
:1037800040F0BB800D9B01330493039E099F0125EC
:1037900007E0594600230A22504601F035FA013568
:1037A000834649465846FFF70FFCAF4200F130030D
:1037B00006F8013BEDDC099A002AC8BF1546039ABA
:1037C000D8BF0125154400220692594601225046D1
:1037D000089301F0F5FB4946834601F069FC002897
:1037E00040F3C88115F8013C039A013D04E0AA4268
:1037F00000F0DA8115F8013D392B05F10108F6D00A
:1038000001332B704946504601F0F4F95CB1069B38
:103810002BB1A34203D01946504601F0EBF92146E3
:10382000504601F0E7F95946504601F0E3F900230C
:1038300088F800302A9B049A1A602C9B002B3FF4D6
:1038400094AC0398C3F800801FB0BDE8F08F01234B
:103850000F936B1E002BBFF6FAACC5F101030C935E
:1038600000230893F5E44046FDF7DAFC32463B4678
:1038700004F0ECFC00287FF4D0AC08F1FF33069391
:10388000CBE4BA4B039303981FB0BDE8F08F0C9DB7
:103890000E9C4E461CE7C0F11C000C9B03440C938D
:1038A000089B0344054408934EE70124E6E4C3F172
:1038B000200306FA03F07CE40146504601F020FBA9
:1038C000289B012B814640F3D3810027D9F8103083
:1038D00009EB8303186901F0E7F9C0F1200026E73E
:1038E000214600230A22504601F08EF9139B002B3B
:1038F000044640F30F830D960993002D00F30B81CE
:10390000002F40F014822646049B039F099903F080
:1039100001027B1E1944289B0A92134309910C93C0
:1039200049465846FFF750FB21460490584601F09F
:10393000BFFB324680464946504601F0D9FB049B06
:10394000C26805463033002A41D1014658460893E3
:1039500001F0AEFB29460690504601F04BF9069A5D
:10396000089B1AB90C99002900F0C082791CB8F1A3
:10397000000F0D46C0F29B81289848EA00080A987B
:1039800050EA080800F09381002A00F3EB81099ABD
:103990003B70974200F0EC81594600230A225046C2
:1039A00001F032F9B442834621464FF000034FF054
:1039B0000A02504613D001F027F93146044600238D
:1039C0000A22504601F020F92F460646A8E7014694
:1039D0005046069301F00EF9069B0122C6E701F05E
:1039E00013F92F46044606469AE7289B022B70DC03
:1039F0000E9B002B81D10D9B494601335846049301
:103A0000FFF7E2FA039D00F13003002205F8013BC5
:103A10000692DAE64946584601F04AFB0028BFF60E
:103A2000A9AE594600230A22504601F0EDF80D9B3D
:103A30005E1E0E9B8346002B7FF452AF139B002B20
:103A400040F360820D9A049209939EE6484B0393DB
:103A500003332EE41C2020E7DDE9041200297FF463
:103A600060AEC2F31303002B00F00D81049F59E6F2
:103A700001230E93299B0D9A134413930133012BB9
:103A80001D460993B8BF01250021172DCAF844101F
:103A90007FF75FAC012204235B0003F11400A8420E
:103AA000114602F10102F7D9CAF8441051E401238A
:103AB0000E93299B002B53DD139309931D46E3E7D7
:103AC00000230E93D6E700230E93F2E7139B09938E
:103AD0000D96099B002B7FF46AAD4946052250469E
:103AE00001F092F801468146584601F0E1FA0028BB
:103AF0007FF75DADDDF80C800D9F312308F8013BA9
:103B000001377B1C49465046049301F073F8002CA2
:103B10007FF485AE87E621462A46504601F050FAEA
:103B20000446EDE6A9EB0606C2E5214632465046BC
:103B300001F0E6F95A4601460446504601F032F9D2
:103B400059468346504601F055F8D9E5DDE90A2388
:103B50004FF00208CDE9102329E4C0F13C009CE6B7
:103B6000012329930993FFF7EFBB00BF988400005E
:103B7000F884000003D1089BDB073FF533AEA8466D
:103B800015F8013D302BFAD03CE6129A002A00F0DD
:103B90004C8103F23343089A1A4408920C9A154652
:103BA0001A440C924E468EE5049B039A013304930B
:103BB0003123137026E64046FDF732FB32463B4682
:103BC000FDF798FBB84B0022FDF7DEF9A1F1507329
:103BD000CDE914011593B54B394600223046FDF767
:103BE000D1F9DDE914783A46434604460D4604F01F
:103BF00055FB002840F066813A4608F10043204614
:103C0000294604F02DFB00283FF4AAAC4FF0000930
:103C10004C46CCE40F9020E600F032810D9AA44B84
:103C2000544204F00F0203EBC203D3E90023DDE9A1
:103C30000A01FDF75FFB241106460F4600F0728172
:103C40009C4D00234FF00208E20706D5D5E900237A
:103C5000FDF750FB08F101080123641005F1080588
:103C6000F2D1002B3FF4BDAB06460F46FFF7B9BBC0
:103C7000049B002B7FF429AEDDE90412C2F3130389
:103C8000002B7FF422AE8C4F1740002F3FF44AAD3B
:103C90000C9B01330C93089B01330893012741E5EA
:103CA00059464A46504601F02BF983462CE5002A36
:103CB000884612DD594601225046069301F080F9EC
:103CC0004946834601F0F4F90028069B40F303813E
:103CD000392B00F0E080049B31333B700D9B069440
:103CE0000133049334468DE55F46DDF818A0DDF816
:103CF00010B00D9B0133049302461C460B46FDF7A2
:103D000043F902460B46CDE9062342464B4604F0F2
:103D1000C5FA40B9DDE9060142464B4604F096FA81
:103D200018B1F90701D5039A0AE4B0467BE561684A
:103D3000504600F039FF0546002800F0F78023695F
:103D400002339A0004F10C010C30FDF709FD2946FD
:103D50000122504601F034F90646D5E50C9B099A3C
:103D60009D1AB0E4392B884600F095800133B4E702
:103D70000D9A069401320492344626E5594650467F
:103D800001F0BEF88346BFE4DDE91823DDE9160142
:103D9000FDF7B0FA039A149B1370109B012BCDE929
:103DA000140100F0B580109E039B1E44434B00227B
:103DB00020462946FDF79EFA0D46044604F08EFA89
:103DC0000746FDF72DFA303702460B4620462946B6
:103DD000FDF7D8F808F8017BB04504460D46E5D15B
:103DE000DDE91478364B002238464146FDF7CCF821
:103DF00022462B4604F034FA002867D13A4643465F
:103E00002F490020FDF7BEF822462B4604F046FA63
:103E100000283FF4A5ABB046013E18F8013C302B1A
:103E2000F9D01A9B01330493FDE41C9BC3F13603C4
:103E3000B1E6099B002B3FF4BEAE139B002B7FF72E
:103E40008FAB0D9A1093013A1C4B1A923046002208
:103E50003946FDF74FFA06460F4608F10100FDF717
:103E6000DFF932463B46FDF745FA0F4B0022FDF7DE
:103E70008BF8A1F15073CDE914011593FFF7D4BA73
:103E8000DDE90A674FF00208FFF7ABBA01343123CE
:103E9000FFF75DBB7D1C0D9B069401330493392312
:103EA00034463B70A0E400BF00001C4000001440FA
:103EB00020860000F88500000000F07F000024400C
:103EC0000000E03F4FF000094C4613E61A9C039AAD
:103ED0000134FFF735BB7FF400AFDA077FF5FDAEA5
:103EE000F6E6DDF858B0DDF860A09AE7392B4246D7
:103EF000D0D0002AC8BF049BB846C8BF313308F8E9
:103F0000013BEBE6289B022B3FF7E0AD0D9672E5F7
:103F1000464665E7289B022B3FF7D8AD139B0D96CD
:103F20000993EAE44FF00208FFF75BBA134B144819
:103F30002A4640F2EA2102F0DFF80024CAF84440A1
:103F40002146504600F030FE039050B90B4B0C4810
:103F500000224FF4D57102F0CFF80A4B0393FFF71C
:103F600004B9039BCAF840304FF0FF331393099311
:103F7000012329940E93FFF7F3BA00BFFC840000DD
:103F800010850000EC840000B1F90C20F8B50C4657
:103F90001107074643D4636842F40062002BA281F4
:103FA0005ADDA56A002D55D000233E683B6093B2D0
:103FB00012F48052E16953D101233846A847421CCC
:103FC00064D0A389A56AE1695B0705D56368C01A57
:103FD000236B0BB1E36BC01A024600233846A84797
:103FE000451C46D13A68B4F90C30002A5AD01D2A33
:103FF00001D0162A39D12269226023F400630021FE
:104000006160A381216B3E6021B304F140039942BA
:1040100002D0384600F030F900202063F8BD266950
:10402000C6B193B22568266099070CBF6369002367
:10403000AD1BA3600CE0D4F824C0E1692B463246E6
:104040003846E047B0F1000CA5EB0C05664409DDED
:10405000002DF0DC0020F8BDE36B002BA1DCF9E7BC
:10406000206DB1E7A3894FF0FF3043F04003A381F7
:10407000F8BDB4F90C302269226023F400630022F9
:104080006260DA04A381BDD52065BBE73B68002BE5
:1040900097D01D2B0FD0162B0DD0A38943F04003D2
:1040A000A381F8BD23F400636260A38122692260CA
:1040B000DB04A7D5E8E73E60CCE700BF38B50D4686
:1040C000044608B1836B1BB1B5F90C0030B938BD9B
:1040D00000F07CF8B5F90C000028F8D029462046FD
:1040E000BDE83840FFF750BF014900F0C1B900BF3B
:1040F000E16100002DE9F84F2D4A4668C2630024B3
:104100000323C0E9B843074600F53B720423C0F817
:10411000E8222146C6E902430822C6E90044C6E96E
:1041200004443466B46106F15800FDF7B3FBDFF8D0
:1041300084B0BD68DFF880A0DFF88090DFF8808071
:10414000204BC6F824A0C6E9076BC6F82890C6F82D
:104150002C800822EB60C5E90044C5E904442C66C4
:10416000AC60AC61214605F15800FDF793FBC5E951
:10417000075BC5E909A9C5F82C80FD68124BEB6007
:10418000C5E90044C5E904442C66AC60AC61214635
:10419000082205F15800FDF77DFB0123C5E9075B07
:1041A000C5E90A98C5F824A0BB63BDE8F88F00BF35
:1041B000E9400000B5530000D95300001954000035
:1041C000395400000900010012000200836B03B1A2
:1041D0007047FFF78FBF00BFF8B5244F0C46064667
:1041E00000F0DEFCBB685D68C4F57E610F3125F030
:1041F00003054B1923F47F6323F00F03A3F58054C9
:10420000B4F5805F07DB0021304601F07BF8BB6826
:104210002B44984204D0304600F0C4FC0020F8BD86
:104220006142304601F06EF801300DD0104ABB6893
:104230002D1B45F001055D60136830461B1B1360A4
:1042400000F0B0FC0120F8BD0021304601F05AF822
:10425000BA68831A0F2BDEDD43F001035360054B70
:1042600003491B68C01A0860D5E700BF200400207E
:10427000F80900202808002000295FD0F8B50C4676
:10428000064600F08DFC54F8043C764FA4F1080576
:1042900023F001016A18D7F808C05068944520F04F
:1042A000030000F08680DB07506002EB000C33D483
:1042B00054F8084CDCF804302D1B2144AC6807F19D
:1042C000080C644503F0010363D0D5F80CE0C4F892
:1042D0000CE0CEF80840002B00F08F8041F0010385
:1042E0006B601160B1F5007F31D27868CB08012294
:1042F000490901338A40024357F833107A6007EBCB
:10430000C302083AC5E9021247F83350CD6030467F
:10431000BDE8F84000F046BCDCF80430DB070ED402
:10432000014407F1080C9368634541F001006CD02B
:10433000D268DA60936068606950D3E7704741F0F3
:104340000103B1F5007F44F8043C1160CDD3B1F511
:10435000206F4FEA512345D28B0903F1390003F155
:104360003802C300F818FB580838984254D05A68ED
:1043700022F003028A4202D99B689842F7D1D8689A
:10438000C5E902308560DD603046BDE8F84000F0E8
:1043900009BC002B61D1D2E902230844D3609A60A2
:1043A00040F001036B6028503046BDE8F84000F053
:1043B000F9BBDA07084407D454F8083CED1A18444E
:1043C000D5E90223D3609A6040F001036B60264B6D
:1043D000BD601B6883429AD8244B30461968FFF7AA
:1043E000FBFE94E7142B0AD9542B1DD80B0B03F1B9
:1043F0006F0003F16E02C300B4E7014493E703F1D9
:104400005C0003F15B02C300ACE7C7E90455C5E9F2
:1044100002CC686069507AE779689210012404FA46
:1044200002F20A437A60ABE7B3F5AA7F06D8CB0B5A
:1044300003F1780003F17702C30093E740F254528E
:10444000934206D88B0C03F17D0003F17C02C3007C
:1044500088E74FF47E737E2284E741F001036B60AE
:10446000116054E7200400202C080020280A0020B6
:104470002DE9F8430746884600F538764FF00009E5
:10448000D6E90154013D11D4A389012B05F1FF3573
:1044900008D9B4F90E300133214603D03846C0475D
:1044A00049EA00096B1C04F16404EDD13668002E62
:1044B000E6D14846BDE8F88300487047200900204F
:1044C0002DE9F0418B890C46990796B008D504F187
:1044D00043030122C4E90432236016B0BDE8F08131
:1044E000B4F90E100029064627DB6A4601F032FFB8
:1044F000002821DB019D05F47045A5F50055B5FAAE
:1045000085F54FF480686D094FF4006741463046E9
:1045100000F046F8B4F90C30F0B1204AF26343F0F1
:104520008003C4F81480A3812060206135BB3B4325
:10453000A38116B0BDE8F081A38913F0800519D0DE
:104540004FF040084146304600F02AF80025B4F903
:104550000C302F460028E0D19A05BED423F0030387
:1045600004F1430243F002030121C4E90421A381C1
:104570002260B2E74FF480682F46C7E7B4F90E1007
:10458000304602F081F810B9B4F90C30CFE7A389B6
:1045900023F0030343F001031BB2C8E7E940000026
:1045A0002DE9F04F01F10B06162E83B0054624D8F5
:1045B000102900F2A38000F0F3FA102618224FF021
:1045C000020CB04F3A44A2F1080354689C4200F038
:1045D000A2806368E268A16823F003032344CA60F1
:1045E00091605A6842F0010228465A60083400F08F
:1045F000D9FA204603B0BDE8F08F36F007067DD427
:10460000B1427BD800F0CCFAB6F5FC7FC0F09881BF
:10461000730A7AD0042B00F26481B30903F1390CD8
:1046200003F138044FEACC03964F3B44A3F1080052
:104630005B68984206D10CE0002980F21481DB68A7
:10464000984206D05A6822F00302911B0F29F3DD2D
:10465000A4463C69DFF83082444568D0616821F0A7
:1046600003018B1B0F2B00F37A81002BC7E9048811
:1046700080F26B81B1F5007F80F01281CB08786801
:104680000133490901228A40024307EBC30157F86D
:104690003300A0600839E1607A6047F83340C460B5
:1046A0004FEAAC0301209840904247D8104206D10F
:1046B0002CF0030C400010420CF1040CFAD007EB74
:1046C000CC0A5346E146D9680EE04A6822F003025C
:1046D000A2EB060EBEF10F0F0C46C96800F30E8167
:1046E000BEF1000F80F21F818B42EED109F101096A
:1046F00019F0030F03F10803E5D165E100240C2351
:1047000020462B6003B0BDE8F08F4FF400734FF0EC
:10471000400C3F2488E7D468A24208BF0CF1020C89
:104720007FF457AF3C69DFF86081444596D17A68E1
:104730004FEAAC03012098409042B7D9BC68636847
:1047400023F003094E4503D8A9EB06030F2B7ADCAF
:10475000DFF838B14E4BDBF800201B6801323344E0
:1047600004EB090A00F0468103F580530F3323F46C
:104770007F6828F00F084146284600F0C3FD411C21
:10478000024600F00581824500F20081414B196824
:1047900041441960084600F06281DBF80010019383
:1047A00001311BBFA2EB0A010918CBF800201960E8
:1047B00012F0070B00F02A81CBF108010A44CBF577
:1047C000805190440831A1EB0801C1F30B0A514616
:1047D0002846009200F096FD421CDDE9002300F01F
:1047E0006481801A00EB0A081968BA6048F0010079
:1047F0005144BC425060196000F03D81B9F10F0F87
:1048000040F23B816068A9F10C0C2CF0070C00F021
:10481000010040EA0C0060604FF0050E04EB0C0054
:10482000BCF10F0FC0E901EE00F247815068144659
:10483000194B1A688A4238BF1960184B1A688A42A5
:1048400038BF1960A6E0A21943F0010346F0010643
:1048500066602846BA60536000F0A4F90834204628
:1048600003B0BDE8F08FD3E902411A44E1608C60E7
:10487000516841F001012846516003F1080400F03D
:1048800091F9B6E620040020280400202808002022
:10489000280A0020F8090020200A0020240A00200D
:1048A000B1F5206F4FEA51226AD3142A00F2BF807B
:1048B00002F15C03DB005B32F818FB5808389842C1
:1048C00000F09B805A6822F003028A4202D99B685A
:1048D0009842F7D1D8687A68C4E902308460DC6015
:1048E000DEE6142B64D9542B00F2A980330B03F1BC
:1048F0006F0C03F16E044FEACC0395E62846A568D9
:10490000A31946F001066660E9608D604EF0010172
:10491000C7E90433C3E90288596044F802E000F0B3
:1049200041F9083465E622442846536843F0010300
:10493000536054F8083FD9608B6000F033F958E6B3
:104940004FEAD60C06F108023BE6214428464B68A4
:1049500043F001034B60083400F024F949E6A21942
:10496000284646F0010643F001056660C7E90422C7
:10497000C2E902885560635000F014F9083438E643
:104980008A0902F13903DB00383295E7BC4261D075
:10499000BC68606820F003084645A8EB060302D80F
:1049A0000F2B3FF750AF284600F0FCF8002420E61C
:1049B00003F15C0C03F15B044FEACC0334E65AF8D4
:1049C0000839534540F098801CF0030F0CF1FF3C70
:1049D000F5D17B6823EA00037B60400098423FF6F4
:1049E000ADAE18B9AAE6400009F104091842FAD0A0
:1049F000CC4664E603F11008BDE6796892104FF0EA
:104A0000010E0EFA02F20A437A6065E702EB080132
:104A10004942C1F30B0A51462846009200F072FC4D
:104A2000431CDDE900237FF4DCAEDA46DCE6542AE1
:104A300026D80A0B02F16F03DB006E323CE7B3F5B8
:104A4000AA7F26D8F30B03F1780C03F177044FEA21
:104A5000CC03E9E5294B1868404418609DE6CAF389
:104A60000B0CBCF1000F7FF498AEBC68C84448F052
:104A700001006060DCE61446DAE60123536092E749
:104A8000B2F5AA7F24D8CA0B02F17803DB00773293
:104A900012E740F25452934224D8B30C03F17D0C38
:104AA00003F17C044FEACC03BEE5ABF1080BD8441C
:104AB000A8EB02084FF0000A96E604F10801284628
:104AC0000093FFF7D9FBBC68009B60681968AFE6EC
:104AD00040F254539A420BD88A0C02F17D03DB005A
:104AE0007C32E9E64FF47E734FF07F0C7E249BE529
:104AF0004FF47E737E22DFE67B686EE7F8090020C4
:104B000001F0FF01102A2BDB10F0070F08D010F87E
:104B1000013B013A8B422DD010F0070F42B3F6D182
:104B2000F0B441EA012141EA014122F007047FF09B
:104B300000070023F0E80256083C85EA010586EAF2
:104B4000010685FA47F5A3FA87F586FA47F6A5FA2E
:104B500087F68EB9EED1F0BC01F0FF0102F007023A
:104B600032B110F8013B013A83EA010313B1F8D1E5
:104B70000020704701387047002D06BF35460338C6
:104B8000073815F0010F07D1013015F4807F02BFFF
:104B9000013015F4C03F0130F0BC0138704700BF50
:104BA000704700BF704700BFC36C70B505460C4628
:104BB0004BB153F8240080B1026843F8242000234D
:104BC000C0E9033370BD2122042101F0B5FA034688
:104BD000E8640028EDD1002070BD012101FA04F63F
:104BE000721D9200284601F0A7FA0028F3D0C0E910
:104BF0000146E4E731B1C36C4A6853F8220008600B
:104C000043F82210704700BF2DE9F0410D690746B7
:104C10000E461C4601F1140E0020DEF800108BB287
:104C200002FB03434FEA134C090C02FB01CC013099
:104C30009BB203EB0C4385424EF8043B4FEA1C4405
:104C4000EBDC3CB1B368AB4207DD06EB8503013515
:104C50005C6135613046BDE8F081716838460131EC
:104C6000FFF7A2FF8046A8B13269023206F10C01BB
:104C700092000C30FCF774FDFB6C726853F8221044
:104C8000316043F82260464606EB850301355C61DE
:104C90003561DFE7024B03484246B52101F02CFAAB
:104CA000FC84000080850000020C12040346CAB98F
:104CB0000304102013F07F4F04BF1B02083013F0D1
:104CC000704F04BF1B01043013F0404F04BF9B0022
:104CD0000230002B05DB13F0804F00F1010008BF0C
:104CE000202070470020E5E7036813F00702014623
:104CF00007D0DA071FD4980721D55B080B60012085
:104D0000704798B2A0B11046DAB20AB908301B0A4F
:104D10001A0704BF1B0904309A0704BF9B0802301E
:104D2000DA0703D45B0800F1010006D00B6070477E
:104D30001B0C1020E8E700207047202070479B08DC
:104D40000B600220704700BF38B5C36C04460D46A7
:104D50004BB15868B0B102685A6000220123C0E923
:104D60000435C26038BD2122042101F0E5F9034673
:104D7000E0640028EDD1094B094800224FF4A071EE
:104D800001F0BAF91C220121204601F0D5F90028D2
:104D9000F1D001220223C0E90123DEE7FC840000F8
:104DA000808500002DE9F04F0E691569AE4285B08F
:104DB0008846144605DB2A46234635460C461646E9
:104DC0009846A3686168AF19BB42B8BF0131FFF7CD
:104DD000EBFE0190002800F08780019B03F114098D
:104DE00009EB870AD14505D24B46002243F8042B34
:104DF0009A45FBD808F1140808EB860B04F114035C
:104E0000D8451A4603EB85055FD22B1B153B23F0D3
:104E1000030304331534A54238BF0423CDE902A7A8
:104E2000AC461F46924605E0090C29D1C34509F15D
:104E3000040948D958F8041B8DB2002DF4D0564609
:104E40004C46002356F8041B22681FFA81FE90B2DC
:104E5000090C05FB0E00120C034405FB012202EBBA
:104E600013429BB243EA0243B44544F8043B4FEA81
:104E70001243E7D849F8073058F8041C090CD5D07C
:104E8000D9F8003050461A464C4600260588120CC8
:104E900001FB052216449BB243EA064344F8043B57
:104EA00050F8045B22682D0C93B201FB053303EB31
:104EB000164384454FEA1346E8D8C34549F80730FE
:104EC00009F10409B6D8DDE902A7002F02DC05E0EC
:104ED000013F03D05AF8043D002BF9D0019B18463E
:104EE0001F6105B0BDE8F08F034B0448019A40F202
:104EF0005D1101F001F900BFFC8400008085000015
:104F000012F003032DE9F0411446064632D10D4656
:104F1000A41020D0D6F84880B8F1000F33D0E307B2
:104F20004FF0000707D4641015D0D8F80000A8B1DE
:104F30008046E307F7D5424629463046FFF732FF61
:104F4000B5B16968F36C641053F821202A6043F806
:104F500021500546E9D12846BDE8F0814246414648
:104F60003046FFF71FFFC8F8000007608046E0E703
:104F70000546D8E7013B0F4A52F823200023FFF7EC
:104F800043FE0546C4E701213046FFF70DFE80468B
:104F900040B1012340F27122C0E904320023B06421
:104FA0000360BCE7044B054842464FF4A07101F092
:104FB000A3F800BFE8860000FC84000080850000A4
:104FC0002DE9F0470C4690462669A368496806EB30
:104FD0006216751C9D4207464FEA621904DD5B00AC
:104FE0009D4201F10101FADC3846FFF7DDFD844600
:104FF000002851D0B9F1000F00F114000EDD09F1C5
:1050000005024FEA820E03460CEB8202002143F8B0
:10501000041B9342FBD1AEF114031844216904F13F
:10502000140318F01F0803EB81012DD0C8F12009EB
:1050300086464FF0000A1A6802FA08F242EA0A02AB
:105040004EF8042B53F8042B994222FA09FAF2D8AD
:105050000B1B153B23F00303043304F115029142AB
:1050600038BF0423BAF1000F18BF2E4640F803A042
:10507000FB6C6268CCF8106053F822102160604627
:1050800043F82240BDE8F087043853F8042B40F879
:10509000042F9942F9D8EBE7034B0448624640F2EB
:1050A000D91101F029F800BFFC84000080850000C0
:1050B0000B6984460069C01A15D10CF1140C143127
:1050C0000CEB830210B401EB830301E0944508D29A
:1050D00052F8044D53F8041D8C42F7D004D24FF01F
:1050E000FF3010BC70477047012010BC704700BFF4
:1050F0002DE9F84F0F691369FF1A002F0E469046ED
:105100007FD101F11405143202EB830205EB830316
:1051100001E09D4278D253F8041D52F8044DA1429B
:10512000F7D069D37168FFF73FFD8146002877D03B
:105130003569D8F81020C76008F1140E06F1140084
:1051400009F1140A06F110010EEB820200EB85074B
:1051500056464FF0000C5EF8044B51F804BFA3B262
:105160001CFA8BFCACEB03034FEA144CCCEB1B4C4E
:105170000CEB234C9BB243EA0C43724546F8043BCC
:105180004FEA2C4CE7D8A2EB0801153908F11508B5
:10519000424521F0030404F1040438BF04242044F0
:1051A00021F0030238BF002287425244544418D9E8
:1051B0002646014651F8043B1CFA83FC4FEA2C4278
:1051C00002EB13421FFA8CFC4CEA02438F4246F872
:1051D000043B4FEA224CEDD8013F3F1A27F003076A
:1051E000E21923B952F8043D013D002BFAD0C9F869
:1051F00010504846BDE8F88F33460127464698468A
:1052000090E7F9DB00278DE70021FFF7CDFC814611
:1052100068B101220023C9E904234846BDE8F88F9C
:10522000064B07484A464FF4107100F065FF034BE8
:1052300003484A4640F2322100F05EFFFC84000041
:105240008085000070B5012182B016461D46FFF72B
:10525000ABFC0446002849D02B46C5F30A55C3F3DE
:1052600013030DB143F48013002E019314D101A850
:10527000FFF73AFD019B636101212030216115B3E5
:10528000069BA5F2334505441D60079BC0F1350020
:105290001860204602B070BD68460096FFF724FDF6
:1052A000019B00B30099C0F1200203FA02F20A4305
:1052B000C34001936261002B14BF02210121A3614D
:1052C0002161002DDCD104EB8102A0F23243106990
:1052D000069A1360FFF7E8FC079BC0EB41101860CB
:1052E000204602B070BD009A6261E4E7034B0448B7
:1052F000224640F20A3100F0FFFE00BFFC840000AD
:105300008085000038B5074D0022044608462A6013
:10531000FBF704F8431C00D038BD2B68002BFBD0F2
:10532000236038BD2C0A002038B5154B1F281D6896
:1053300020D8D5F8DC22044662B152F820304BB1B7
:10534000012B15D0591C0FD0002542F8205098474A
:10535000284638BD284600F02BF82246014628464C
:10536000BDE8384000F00EB816232B60012038BD90
:10537000002038BD16232B604FF0FF3038BD00BF32
:105380000000002070B50C46084D0346002620465C
:1053900011461C462E60FAF7E5FF431C00D070BD95
:1053A0002B68002BFBD0236070BD00BF2C0A0020AF
:1053B000FAF7D9BF10B50C46B1F90E1001F024FA76
:1053C000002803DB236D0344236510BDA38923F468
:1053D0008053A38110BD00BF2DE9F0410C46B1F907
:1053E0000C101F46CB05054616460BD421F4805100
:1053F000A1813B46B4F90E1032462846BDE8F04183
:1054000000F064BEB4F90E100223002201F054F93A
:10541000B4F90C10EAE700BF10B50C46B1F90E1054
:1054200001F04AF9A389421C0EBF23F4805343F4D0
:1054300080532065A38110BDB1F90E1000F0B8BEF5
:1054400010B4044C84461346206810BC0A466146DA
:1054500000F03CBE000000202DE9F84F0B6E9C04CC
:1054600090462DD59368126843B38B46064602F1E9
:10547000080959E9025A5FEA9A0715D0043D002449
:1054800001E0A7420ED055F8041F5A46304600F0FE
:105490004FFF431C04F10104F3D10023C8E9013399
:1054A000BDE8F88FD8F808302AF0030AA3EB0A0306
:1054B000C8F8083009F10809002BDAD10020ECE720
:1054C00000F05EFF0023C8E90133BDE8F88F00BF9C
:1054D00010B4946814B110BCFFF7BEBF20465460EE
:1054E00010BC70472DE9F04FABB01C4688461746FC
:1054F0000693834618B1836B002B00F0C681B8F980
:105500000C1088048AB20AD4D8F8603041F40051F3
:1055100023F40053A8F80C108AB2C8F860301107C1
:1055200040F1A680D8F81030002B00F0A18002F0E6
:105530001A020A2A00F0AA801AAB0D930023CDE9C3
:105540000E3309930DF1680904933B78002B00F0AA
:10555000C9803C4604E014F8013F002B00F0A48011
:10556000252BF8D1E51B40F0A1802378002B00F01B
:10557000B980002101344FF0000327468DF82F3009
:1055800008464FF0FF3A0D460C4617F8012BA2F1E2
:105590002003582B00F2B380DFE813F06302B10060
:1055A000B1006002B100B100B100B100B100B100C2
:1055B0007A018F04B10082018501B10074025900A3
:1055C0005900590059005900590059005900590013
:1055D000B100B100B100B100B100B100B100B10043
:1055E000B100B1006902B100B100B100B100B10079
:1055F000B100B100B100B100B1002D02B100B100A5
:10560000B100B100B1002502B100B1001E02B1002D
:10561000B100B100B100B100B100B100B100B10002
:10562000B1000E024E01B100B100B1005D024E01A9
:10563000B100B1006700B10048023602FF01670007
:10564000B100DF01B100D001B100B1009C01A2F1B5
:105650003003002417F8012B04EB840403EB44040B
:10566000A2F13003092BF5D991E745F010058CE73D
:1056700041465846FDF71EFC002840F08A84B8F8E1
:105680000C2002F01A020A2A7FF456AFB8F90E3045
:10569000002BFFF651AF23463A46414658462BB001
:1056A000BDE8F04F00F088BCE51B1BD00E9B0F9AA5
:1056B00001332A44072BC9E900750F920E9305DCCC
:1056C00009F10809049B2B4404934EE7002A00F0DB
:1056D0009E830DAA41465846FFF7BEFE30B90DF134
:1056E0006809EFE70F9B002B40F02484B8F80C30DA
:1056F0005B0600F14E8404982BB0BDE8F08F059452
:10570000002940F01384002AECD04FF000038DF8FC
:105710002F3001238DF840200193039310AC0295A4
:105720004FF0000A029B13F00203079302D0019B83
:1057300002330193DDE90E2C029B501C13F084030D
:105740000146089305D1059B019D5D1B002D00F3CB
:10575000A7829DF82F0090B10DF12F020CF1010CE2
:10576000C9F8002007294FF00102CDE90E1CC9F845
:10577000042000F376820A4609F108090131079BEB
:10578000EBB10CAB0CF1020CC9F8003007294FF05B
:105790000203CDE90E1CC9F8043040F37C82BCF151
:1057A000000F00F02F830DAA41465846FFF754FE24
:1057B00000289BD1DDE90E2C0DF16809511C089BD6
:1057C000802B00F0A881039BAAEB0306002E00F3B8
:1057D000FE81039AC9F8004002EB0C030729CDE9CA
:1057E0000E13C9F8042040F37F81002B00F09E8245
:1057F0000DAA41465846FFF72FFE00287FF476AFEA
:105800000F9B0DF16809029A520705D5059A019977
:10581000541A002C00F39582DDE90421019881429D
:10582000ACBF521812180492002B40F00C820023D7
:105830000E930DF1680988E60594002940F0A083D5
:10584000069BEE0653F8042B069302D46C0600F177
:1058500020831346002AC0F2E882BAF1FF3F9DF888
:105860002F1006D025F080000290002A00F0D3828D
:10587000029D092B00F2EE8230338DF86730012350
:10588000029503930DF167041BE1FEF79FFC36E6DA
:10589000069B53F8044B002C80F2F182644206937D
:1058A00045F0040571E617F8012B2A2A00F07683EB
:1058B000A2F13003092B4FF0000A3FF668AE17F84B
:1058C000012B0AEB8A0A03EB4A0AA2F13003092BE7
:1058D000F5D95CE60594002940F04683944B099382
:1058E0000699EC0651F8043B069102D4680648BFBD
:1058F0009BB2E90702D5002B40F0CE8202220021A4
:10590000BAF1FF3F8DF82F1000F0C08025F0800025
:105910000290002B40F0B980BAF1000F40F0E78010
:10592000002A40F07C8215F00103039300F0AA8264
:1059300030238DF867300DF16704C2E0059400292B
:1059400040F01583069A52F8043B0692EA0602D408
:105950006E0648BF9BB20122D1E7069E059456F819
:10596000044B4FF000038DF82F30002C00F0C7825D
:10597000BAF1FF3F00F0AC82524600212046FFF70B
:10598000BFF8002800F0DF82031B9DF82F1003935F
:10599000069602954FF0000A93E0069A059452F895
:1059A000043B069247F63002ADF83020604A099277
:1059B00045F002050222A2E7069B05944FF0000283
:1059C0008DF82F2053F8042B069301238DF84020E7
:1059D0000193039310ACA2E60594002940F0CA821B
:1059E000544B09937CE7069A059452F8043B0692BF
:1059F00045F01005AFE7069A059452F8043B06926D
:105A000045F0100500227AE70594002940F0A382B2
:105A1000069A15F0100152F8043B0692F2D115F0E7
:105A200040023FF46CAF9BB20A4668E7002940F0A1
:105A30009582069AE80602F1040307D46906069ADD
:105A400004D512680499118006937EE512680499C2
:105A50001160069379E545F0400596E545F00105AE
:105A600093E500287FF491AD012120208DE5059478
:105A7000002940F07682069B53F8042B069345F0EC
:105A80001005E6E645F080057FE5029D012A3FF41A
:105A9000F0AE022A31D01AAC03F007023032DB0834
:105AA000204604F8012DF7D1EE072FD5302A2DD04E
:105AB0003023023804F8013C1AAB1B1A02950393F9
:105AC0000446039B5345B8BF5346019300293FF456
:105AD00029AE0133019325E6039B1A9401221B93FF
:105AE0000F930E920DF1680909F108098BE6012A5E
:105AF00000F02782022A029DCDD109981AAC03F04A
:105B00000F021B09825C04F8012DF8D11AAB1B1B94
:105B100002950393D5E7059B01981E1A002E7FF787
:105B200052AE102E40F33282034D63460DE000BFAB
:105B30007C8400006884000004870000911C09F147
:105B400008090246103E102E1DDD501C1033102196
:105B50000728CDE90E03C9F80050C9F80410EDDD9F
:105B60000DAA002B78D0414658460DF16809FFF781
:105B700073FC00287FF4BAADDDE90E23103E102E31
:105B800002F10101E1DC08469C46B4440728CDE956
:105B90000E0CC9F80050C9F8046040F37581BCF1DF
:105BA000000F00F0B5810DAA41465846FFF754FC9E
:105BB00000287FF49BAD039BDDE90E2CAAEB0306C6
:105BC000002E02F101010DF168097FF702AE102EDF
:105BD000BC4D25DD4FF0100A634606E0911C09F12B
:105BE00008090246103E102E19DD501C10330728FC
:105BF000C9E9005ACDE90E03F0DD0DAA4146EBB12B
:105C000058460DF16809FFF727FC00287FF46EADB8
:105C1000DDE90E23103E102E02F10101E5DC9C4669
:105C2000B4440729CDE90E1CC9F80050C9F8046036
:105C300000F3D28009F108090131CAE501211A46B1
:105C40000DF16809CEE70DAA41465846FFF704FC5E
:105C500000283FF4ECAD49E501211A460DF1680931
:105C600070E7BCF1000F00F0CA800DAA414658460B
:105C7000FFF7F2FB00287FF439ADDDE90E2C0DF1C2
:105C80006809511C7BE502231B939C460CAB1A93BD
:105C900001210DF168090A4609F10809511C8EE538
:105CA000102D40F36A814946874EB9461023274696
:105CB000644607E002F1020E08310246103D102D45
:105CC0001ADD501C10340728C1E90063CDE90E0429
:105CD000F0DD0DAA414658461CB3FFF7BDFB002876
:105CE0007FF404ADDDE90E24103D102D02F1010E0C
:105CF0001AA94FF01003E4DCA4463C464F468946FF
:105D0000AC44BEF1070FCDE90EECC9F80060C9F84C
:105D1000045000F38E8009F108090EF1010172466A
:105D200017E522464FF0010E1AA9C7E7029A0E9313
:105D3000510748D5059A0199541A002C43DD0DF1FD
:105D40006809102C0E9940F31E815F4E10250846FD
:105D500006E0811C09F108091046103C102C19DDE1
:105D6000421C1033072AC9E90065CDE90E23F0DD96
:105D70000DAA1BB341465846FFF76EFB00287FF47F
:105D8000B5ACDDE90E03103C102C00F101010DF162
:105D90006809E5DC084623440728C9E90064CDE921
:105DA0000E037FF739AD73B10DAA41465846FFF790
:105DB00053FB00287FF49AAC0F9B2DE50121184678
:105DC0000DF16809C9E7DDE9043201998A42ACBFE7
:105DD0009B185B1804932AE5BCF1000F3FF47CAEDE
:105DE0000DAA41465846FFF737FB00287FF47EACEA
:105DF0000E99DDF83CC001310DF16809E9E4079B1B
:105E0000002B52D1012162460DF16809D7E40E92B0
:105E10000DF1680956E4BAF1000F40F092804FF09E
:105E2000000ACDF80CA01AAC4BE653422D210122FA
:105E300066E5BCF1000F56D00DAA41465846FFF763
:105E40000BFB00287FF452ACDDE90E2C0DF1680944
:105E5000511C7EE41D4E1AACA6FB0302D20802EBD5
:105E60008200A3EB4000303004F8010D18460928E9
:105E70001346F1D81AAB1B1B0295039321E6069338
:105E8000FFF783BB1AAC1CE609F10809411C024666
:105E900099E412B21346DDE48DF8312030228DF8FA
:105EA000302045F00205022229E502231B939C467F
:105EB0000CAB1A930DF16809EEE601212B20FFF7D8
:105EC00064BB00BF04870000F4860000CDCCCCCCBE
:105ED000204606960295FBF753FD4FF0000A9DF809
:105EE0002F100390EDE59DF82F20B2B101210DF1A7
:105EF0002F021B911A920DF168098C463BE4534620
:105F0000062B28BF0623294C03930696019306E42B
:105F1000012162460DF1680955E4079B002B7FF4CF
:105F2000B2AE624601210DF168094CE48DF82F00F4
:105F3000FFF7E9BB0DAA41465846FFF78DFAFFF778
:105F4000D5BB029D98E4CDF80CA09DF82F100696C5
:105F500002958246B5E58DF82F0059E58DF82F00A2
:105F600067E58DF82F0086E58DF82F00B6E48DF8F3
:105F70002F00E7E48DF82F0032E50D4E8646BFE690
:105F80008DF82F005CE40A4E481C04E7094D0846D2
:105F9000FBE54FF0FF330493FFF7ADBB069B53F8CF
:105FA000042B069342EAE27AFFF7EFBA90840000EE
:105FB000F48600000487000070B50C468989ADF5B1
:105FC0008D6D21F00201ADF81010216E1991E1895B
:105FD000ADF81210E1690891616A0A911AA901915C
:105FE00005914FF48061039106910021079101A969
:105FF0000646FFF777FA051E07DB01A93046FEF7D4
:106000005DF8002818BF4FF0FF35BDF810305B0673
:1060100003D5A38943F04003A38128460DF58D6D78
:1060200070BD00BF10B51A4C002924689AB02ADB55
:10603000019005904FF40270ADF8100013D00139B3
:106040004FF6FF7003910691ADF8120001A92046AA
:1060500000F0DCFD421C01DA8B232360019B00224F
:106060001A701AB010BD4FF6FF7003910691ADF88B
:10607000120001A9204600F0C9FD431C01DA8B2360
:1060800023601AB010BD8B2323604FF0FF30F8E778
:106090000000002070B50B4E9AB004466FF000452A
:1060A000CDE90545134601940A463068064C039530
:1060B00001A9049400F0AAFD019B00221A701AB0F5
:1060C00070BD00BF000000200802FFFF38B50C467D
:1060D000084D8446114620461A4600232B6064462C
:1060E00002F02CF9431C00D038BD2B68002BFBD0EC
:1060F000236038BD2C0A002000B50B4C25681446DF
:10610000EE681A4685B003460D464CB10749009526
:10611000CDE901143046064900F0A2F801F0B6FFBF
:1061200004490C46F3E700BF00000020148700007C
:10613000248700002087000038B5A1FB02148CBB27
:10614000FEF72EFA0546E0B150F8042C22F00302C7
:10615000043A242A17D8132A1AD91B2AC0E9004462
:106160001DD9242A14BF00F1100200F118024FF0CB
:106170000003C0E9024404BF04614461C2E9003382
:106180009360284638BD2146FBF784FB284638BD7E
:1061900002460023C2E900339360284638BD00F16F
:1061A0000802F6E700F016F80C2300250360E8E784
:1061B00038B5074D0022044608462A60FAF7BCF8B5
:1061C000431C00D038BD2B68002BFBD0236038BDAA
:1061D0002C0A0020014B1868704700BF0000002007
:1061E00070B539B106460C4608B1836B63B3B4F998
:1061F0000C3013B90025284670BD21463046FDF706
:10620000C3FEE36A054633B1E1693046984700288A
:10621000B8BF4FF0FF35A3891B061CD4216B41B1D9
:1062200004F14003994202D03046FEF725F80023DE
:106230002363616C21B13046FEF71EF800236364CE
:106240000023A381284670BDFDF7C0FFB4F90C30D0
:10625000002BCFD0D1E721693046FEF70DF8DDE7FE
:106260000EB410B583B005AB064C53F8042B019364
:1062700001462068FFF736F903B0BDE8104003B0CF
:10628000704700BF000000202DE9F04383B00746AF
:106290008846144600F00AFA012803D108F1FF33BA
:1062A000FE2B37D9424604F1580301A9384601F0C4
:1062B000C5FE421C064633D038B39DF804C00DF12C
:1062C0000509002509E023685A1C226083F800C0F4
:1062D0000135B54219D219F801CBA368013B002B57
:1062E000A360F0DAD4F818E07345614622463846D8
:1062F00002DBBCF10A0FE6D101F048FE431CE7D1F6
:106300000646304603B0BDE8F0834646304603B04B
:10631000BDE8F0835FFA88FC8DF804C00646CEE73E
:10632000A389304643F04003A38103B0BDE8F08366
:10633000B2F90C3013F4005F0AD110B4146E43F4B8
:10634000005344F400541466938110BCFFF79CBFC3
:10635000FFF79ABF70B50C46084D0346002620464D
:1063600011461C462E60F9F7EAFF431C00D070BDB1
:106370002B68002BFBD0236070BD00BF2C0A0020CF
:106380009368002B00F0FC802DE9F04FB1F90C3040
:106390001FFA83FC1B0783B0904681460C4631D51B
:1063A0000B697BB31CF00207D8F800603AD00027D5
:1063B000D4F824B0E169DFF8CCA23D4655452B4620
:1063C0003A4628BF53464846C5B1D847002840F34F
:1063D000CD80D8F808301B1A07442D1AC8F80830A9
:1063E000002B00F0B98055452B46D4F824B0E16964
:1063F00028BF53463A464846002DE6D1D6E90075F7
:106400000836DBE721464846FCF754FD002840F0FB
:106410003681B4F90C30D8F800601FFA83FC1CF008
:106420000207C4D11CF0010A66D12368A16857464F
:1064300018468B46002F5BD01CF4007F00F0B48020
:10644000B9420A4600F2E0801CF4906F30D0216916
:106450005D1A636903EB430B0BEBDB7B6B1C4FEAB1
:106460006B0B3B445B455A4684BF9B465A461CF423
:10647000806F00F0E88011464846FEF791F800284A
:1064800000F0F7802A4621690190FBF769F9A2899B
:10649000019B22F4906242F08002A2815819ABEB7A
:1064A0000505C4F814B02361A5602060BB463A46D8
:1064B0005146019200F02CF9A1682368019AA1EBE2
:1064C0000B011A443D46A16022600027D8F808302D
:1064D0005B1BAA44C8F80830002B3DD0B4F90CC0AF
:1064E0002368A1681FFA8CFC18468B46002FA3D1A5
:1064F000D6E900A708369BE73846BB463D46002D47
:1065000040D0002845D03A46D4E904C32068A168A9
:10651000AA4228BF2A46604504D901EB030A524526
:1065200000F38280934272DCE169D4F824C05A46B9
:106530004846E047B0F1000A18DDB7EB0A070FD074
:106540000120D8F80830A3EB0A03D344A5EB0A05D1
:10655000C8F80830002BD2D1002003B0BDE8F08F7E
:1065600021464846FDF7AAFD0028EAD0B4F90C30D0
:1065700043F040034FF0FF30A38103B0BDE8F08F3C
:1065800000207047756833460836002DFAD0D3F8DE
:1065900000B02A460A215846FEF7B2FA002865D014
:1065A0000130A0EB0B07AEE722699A4214D362696F
:1065B000BA4211D86FF00043BB4228BF3B46656A20
:1065C00093FBF2F3E16902FB03F348465246A84706
:1065D000051ECBDD7F1B79E7B94228BF39460D4642
:1065E00018460A46514600F093F8A1682368491BF3
:1065F0002B44A16023600029ECD121464846FDF7D9
:106600005DFD0028E6D0B1E7BB463A4650E7594663
:10661000019200F07DF8019AA3689B1AA360236899
:1066200013442360924688E75946524600F070F8BA
:1066300023685344236021464846FDF73FFD002868
:106640003FF47BAF92E7484600F0F4F80346002899
:106650007FF424AF21694846FDF70EFEB4F90C30F3
:106660000C2223F08003C9F8002081E76A1C17463A
:106670004AE70C22B4F90C30C9F8002078E74FF053
:10668000FF306AE700FCFF7F38B5074D0022044663
:1066900008462A60F9F758FE431C00D038BD2B6825
:1066A000002BFBD0236038BD2C0A0020014B93F84F
:1066B000280170473008002038B50C46084D844644
:1066C000114620461A4600232B606446F9F73EFE29
:1066D000431C00D038BD2B68002BFBD0236038BD95
:1066E0002C0A002082B049B15AB16BB113780B600B
:1066F0001278101E18BF012002B0704701A9002AAD
:10670000F3D1104602B070476FF00100F4E700BF0C
:1067100088420DD98B1883420AD900EB020CBAB11A
:10672000624613F801CD02F801CD9942F9D17047C4
:106730000F2A0ED8034602F1FF3C4AB10CF1010CBE
:10674000013B8C4411F8012B03F8012F6145F9D16D
:10675000704740EA01039B0750D1A2F1100370B5C6
:1067600001F1200C23F00F0501F1100E00F11004CF
:10677000AC441B095EF8105C44F8105C5EF80C5CDD
:1067800044F80C5C5EF8085C44F8085C5EF8045C55
:1067900044F8045C0EF1100EE64504F11004E9D152
:1067A000013312F00C0F01EB031102F00F0400EBA8
:1067B000031327D0043C24F003064FEA940C1E4434
:1067C0001C1F8E465EF8045B44F8045FB442F9D1A6
:1067D0000CF1010402F0030203EB840301EB8401DA
:1067E00002F1FF3C4AB10CF1010C013B8C4411F861
:1067F000012B03F8012F6145F9D170BD02F1FF3C77
:1068000003469BE72246EBE738B50C46084D844625
:10681000114620461A4600232B60644601F086FD8F
:10682000431C00D038BD2B68002BFBD0236038BD43
:106830002C0A00202DE9F84F1646002900F09C8014
:106840000C4606F10B050746FEF7AAF9162D54F87B
:10685000040C5DD810252A46AE425ED820F003080D
:106860009045A4F1080963DABC4BD3F808E009EBC2
:10687000080CE645DCF8041000F0948021F00103D8
:1068800063445B68DB076CD421F0030E08EB0E0356
:10689000934248DAC00711D454F8083CA9EB030B23
:1068A000DBF8043023F003018E44C644964580F2A1
:1068B0000F8108EB0103934280F2E48031463846B1
:1068C000FDF76EFE0646E8B154F8043C23F00103E0
:1068D0004B44A0F10802934200F0CE80A8F10402DC
:1068E000242A00F2F180132A00F2A88003462246EF
:1068F000116819605168596092689A60214638465B
:10690000FDF7BAFC3846FEF74DF93046BDE8F88F82
:1069100025F00705002D2A469EDA0C233B60002651
:106920003046BDE8F88F9846DCE90223D3609A60D0
:10693000D9F80430A8EB05020F2A03F0010309EB94
:1069400008001ED848EA0303C9F80430436843F03E
:106950000103436038462646FEF724F93046BDE879
:10696000F88FC307AAD454F8083CA9EB030BDBF853
:10697000041021F003019CE7BDE8F84F1146FDF734
:106980000FBE09EB05012B4342F00102C9F80430A8
:106990004A60436843F00103436008313846FDF71D
:1069A0006BFCD7E721F0030E08EB0E0105F1100C8C
:1069B00061454EDAC10781D454F8081CA9EB010BDC
:1069C000DBF8041021F003018E440EEB080AD445D5
:1069D0003FF76FAF5E46DBF80C1056F8080FA8F1D2
:1069E0000402242AC160886000F2DD80132A40F28C
:1069F000D8802168CBF808106168CBF80C101B2AEE
:106A000000F2E18008340BF1100221681160616826
:106A10005160A16891600BEB0501AAEB050242F001
:106A2000010299604A60DBF8043003F001032B4354
:106A30003846CBF80430FEF7B5F871E723680360F9
:106A4000636843601B2A69D804F1080200F1080357
:106A50004EE709EB05029A604B1B43F001035360BC
:106A600054F8043C03F001032B43384644F8043C3B
:106A7000FEF798F8264653E750F8043C23F003034A
:106A8000984455E75E46DBF80C1056F8080FA8F15D
:106A90000402242AC16088604DD8132A49D921688C
:106AA000CBF808106168CBF80C101B2A58D80834B2
:106AB0000BF1100298462368136063685360A36863
:106AC0009360D946344633E72146FFF721FE15E7A8
:106AD000DCE902135E46CB60996056F8081FDBF8CC
:106AE0000C30CB60A8F10402242A99602DD8132A17
:106AF00029D92368CBF808306368CBF80C301B2AFF
:106B000043D808340BF1100322681A6062685A6097
:106B1000A2689A60F046D946344609E7A3688360C4
:106B2000E368C360242A27D004F1100200F11003A7
:106B3000DEE63246BEE7214630469846D946FFF7A4
:106B4000E7FD3446F4E63346DEE721463046F046BC
:106B5000D946FFF7DDFD3446EAE600BF20040020F9
:106B6000A168CBF81010E168CBF81410242A20D0CB
:106B700010340BF118029DE72369036161694161DB
:106B800004F1180200F11803B2E6A368CBF8103044
:106B9000E368CBF81430242A21D010340BF1180309
:106BA000B2E7324631E721463046FFF7B1FD164BDA
:106BB00031E72269CBF818206269CBF81C20183421
:106BC0000BF1200276E7A168CBF81010E168CBF852
:106BD0001410242A0DD010340BF1180215E7236984
:106BE000CBF818306369CBF81C3018340BF1200354
:106BF0008AE72269CBF818206269CBF81C20183488
:106C00000BF1200201E700BF200400202DE9F04F26
:106C1000BFB08A4690460D930C90FDF74DFC03687B
:106C200015931846FAF7ACFEBAF80C3014901F060C
:106C300004D5DAF81030002B00F090860023CDE95F
:106C40002233129313931693099300240023CDE962
:106C500010342EAA21929146D34698F80030002B8A
:106C600000F03781444604E014F8013F002B00F0A7
:106C70008780252BF8D1B4EB080540F08580237878
:106C8000002B00F026810023621C8DF86730184627
:106C90004FF0FF3519461C46904618F8017BA7F1C6
:106CA0002002582A00F28B80DFE812F09602890059
:106CB000890088028900890089008900890089008B
:106CC0009401470689009C019F018900A802590090
:106CD00059005900590059005900590059005900EC
:106CE000890089008900890089008900890089005C
:106CF000890089009C0225018900250189008900FD
:106D0000890089005802890089006402890089008D
:106D10008900890089005B02890089007D02890061
:106D2000890089008900890089008900890089001B
:106D300089006E026A0125012501250185026A018B
:106D40008900890067008900430231022002670040
:106D50008900FA018900EA0189008900B601A7F1DA
:106D60003002002118F8017B01EB810102EB4101A7
:106D7000A7F13002092AF5D991E744F010048CE715
:106D8000B4EB080500F0A580239B2B442393229BA2
:106D90000133072BC9E90085229305DC09F10809B5
:106DA000099B2B4409936AE70C9821AA594601F0E4
:106DB00075F9002840F04F830DF1B809F0E70B9109
:106DC000002B40F09587002F00F0838000238DF882
:106DD000673001238DF8907007930A9324AD002348
:106DE000069408930F93069B13F0020302D0079AB0
:106DF00002320792069A239C12F084020E9205D169
:106E00000B9A0799561A002E00F388839DF8672085
:106E10008AB1229A0DF1670101320134C9F80010DC
:106E2000072A4FF0010123942292C9F8041000F3BD
:106E3000C98309F1080983B1229B1AAA01330234DC
:106E4000C9F80020072B4FF0020223942293C9F8BF
:106E5000042000F3AB8309F108090E9B802B00F09E
:106E60006682089B0A9AA3EB020ABAF1000F00F3AC
:106E7000A882069BDE0500F1EA810A9BC9F804306E
:106E80001C44229BC9F800500133072B2394229302
:106E900000F3EE8209F10809069B5A0705D50B9B02
:106EA000079A9D1A002D00F39B83099B0B9A079963
:106EB0008A42ACBF9B185B180993002C40F0C38238
:106EC0000023229398F800300DF1B809002B7FF4CD
:106ED000C9AE239BDA46002B40F0B187BAF80C30DC
:106EE00013F0400F099B18BF4FF0FF330993099827
:106EF0003FB0BDE8F08F0B910895002B40F0AA87BA
:106F00000D9B073323F00701F1E8022323F000452E
:106F1000CDE910230D9116461046AA4B29464FF095
:106F2000FF3201F0C5F9002840F09C84A54B3046A3
:106F300029464FF0FF3201F09DF9002840F092847D
:106F4000DDE910010022002301F08AF9002840F059
:106F5000A7869DF867109C4D24F0800306939B4BF9
:106F60000022472FC8BF1D460323CDE907320A93ED
:106F70000F9200293FF437AF079B0133079332E7A5
:106F80000B910895002B40F069870D9BE50653F89F
:106F9000042B0D9302D4600600F160841346002A8E
:106FA000C0F22A8408989DF86710013006D024F0BA
:106FB00080000690002A00F0C283069C092B00F294
:106FC0001C8530338DF8B730012306940A930DF1F8
:106FD000B70533E10D9A52F8041B002980F22A8488
:106FE00049420D9244F0040457E618F8017B2A2F19
:106FF00000F0B087A7F13002092A4FF000053FF6F4
:107000004EAE18F8017B05EB850502EB4505A7F1AF
:107010003002092AF5D942E60B910895002B40F081
:1070200006876B4B13930D9AE10652F8043B0D92C1
:1070300002D4620648BF9BB2E60702D5002B40F09F
:1070400003840222002108988DF86710451C00F087
:10705000D98024F080050695002B40F0D2800028CE
:1070600040F05081002A40F06E8314F001030A932F
:1070700000F0E38330238DF8B7300DF1B705DDE084
:107080000B910895002B40F0E1860D9AE60652F828
:10709000043B0D9202D4600648BF9BB20122D1E7A7
:1070A0000D9E089556F8045B089B0B914FF0000A63
:1070B0008DF867A0002D00F022855A1C00F0868410
:1070C0001A4651462846FDF71BFD002800F0A4860D
:1070D000431B0A9323EAE3739DF86710CDF820A0C1
:1070E0000D9606940793CDF83CA042E70D9A0B91BC
:1070F00052F8043B0D9247F63002ADF86820344A4E
:107100001392089544F00204022278279AE70B9123
:107110000895002B40F0A6860D9A14F0100152F845
:10712000043B0D922ED114F040028BD09BB20A4644
:1071300088E7002B40F09A860D9AE00602F10403DE
:1071400007D461060D9A04D51268099911800D9330
:1071500083E51268099911600D937EE544F00804F7
:107160009BE50D9A0B9152F8043B089544F01004EE
:107170000D9293E70D9A0B9152F8043B089544F059
:1071800010040D9200225DE70D9B0B9100228DF8FB
:10719000672053F8042B0D9301238DF8902007935B
:1071A0000A9324AD1BE60B910895002B40F06286F4
:1071B000084B139337E744F040046EE544F00104B4
:1071C0006BE500BFFFFFEF7F588400005C84000088
:1071D0007C8400006884000000287FF45EAD0123F9
:1071E00020205AE50B910895002B40F024860D9B3A
:1071F00053F8042B0D9344F01004CFE644F08004C0
:107200004BE5069C012A3FF4D9AE022A00F08180AA
:107210002EAD03F007023032DB08284605F8012DB9
:10722000F7D1E3077ED5302A7CD03023023805F829
:10723000013C2EAB1B1A06940A930546089B0A9A3A
:107240009342B8BF1346079300230F9391E6652F2F
:1072500040F31981DDE910010022002300F0F6FF60
:10726000002800F0F881229BB34AC9F800200133BE
:1072700001340122072B23942293C9F8042000F340
:10728000178409F108091B9B129A934203DB069BA2
:10729000DD077FF501AE149B159A1C44C9E9002354
:1072A000229B23940133072B229300F31B8409F1C3
:1072B0000809129B5D1E002D7FF7EEAD102D229B5D
:1072C0009E4E40F3CA80DDF830A0102705E009F19A
:1072D0000809103D102D40F3C08001331034072BF6
:1072E000C9E90067CDE92234F1DD21AA59465046AB
:1072F00000F0D4FE002840F0AE80DDE922340DF12C
:10730000B809E6E7012A00F04C85022A069C7FF4C2
:107310007FAF13982EAD03F00F021B09825C05F8B6
:10732000012DF8D12EAB5B1B06940A9386E70B9BCD
:10733000079AA3EB020ABAF1000F7FF792ADBAF1F8
:10734000100F229B7D4E2EDD32460E955E460C9D23
:10735000BB46174606E0AAF1100ABAF1100F09F170
:1073600008091BDD013310341022072BCDE922342C
:10737000C9F80070C9F80420EDDD21AA314628467D
:107380000DF1B80900F08AFE002840F06281AAF1F0
:10739000100ABAF1100FDDE92234E3DC3A460E9D03
:1073A0005F46B346164601335444072BCDE92234D9
:1073B000C9F80060C9F804A000F3878309F108093F
:1073C0004FE5BAF1100F229B5C4E2EDD3246089538
:1073D0005E460C9DBB46174606E0AAF1100ABAF1BC
:1073E000100F09F108091BDD013310341022072B9F
:1073F000CDE92234C9F80070C9F80420EDDD21AAD6
:107400003146284600F04AFE002840F02281AAF1C9
:10741000100ABAF1100FDDE922340DF1B809E3DCEE
:107420003A46089D5F46B346164601335444072B3F
:10743000CDE92234C9F80060C9F804A000F3CF8177
:1074400009F1080915E50C9821AA594600F026FE15
:1074500000283FF435ADDA4640E501332C44072BD4
:10746000C9F80060C9F80450CDE922347FF712ADA5
:107470000C9821AA594600F011FE0028EBD1239C5C
:107480000DF1B80908E5129B229F012B04F10104BC
:1074900007F1010709F1080A40F35A810123072F78
:1074A000CDE92274C9F80050C9F8043000F3A8816E
:1074B000149B159A01371C44072FCAE90023CDE914
:1074C000227400F3AA810AF1080A129BDDE9100177
:1074D00003F1FF390022002300F0B8FE002840F03D
:1074E0005281013701354C44072FCDE92274CAF887
:1074F0000050CAF8049000F339810AF1080A169B7B
:10750000CAF8043001371C44072F1DABCDE92274A3
:10751000CAF80030ACDC0AF10809BDE4102E229A4A
:1075200035DD59461793B34623462E460C9C4FF043
:10753000100A0D460BE000BF98840000748700001D
:10754000ABF1100BBBF1100F09F1080919DD013285
:10755000BB491033072AC9E9001ACDE92223EFDD20
:1075600021AA294620460DF1B80900F097FD002810
:1075700040F09B82ABF1100BBBF1100FDDE9222331
:10758000E5DC29461C46179B35465E468B46013294
:10759000AB49C9F804603444072ACDE92224C9F86C
:1075A000001000F3738209F108092FE40C9821AA56
:1075B000594600F073FD00287FF44DAF239C0DF178
:1075C000B8094AE40C98179321AA594600F066FDC1
:1075D00000287FF440AF239C179B0DF1B8092AE4E3
:1075E000102D229B1FDD0C9F102604E0103D102D56
:1075F00009F1080917DD0133914A1034072BC9E955
:107600000026CDE92234F1DD21AA594638460DF194
:10761000B80900F043FD00287FF41DAF103D102D88
:10762000DDE92234E7DC0133854AC9F804502C44F3
:10763000072BCDE92234C9F800207FF736AC0C982F
:1076400021AA594600F02AFD00287FF404AF239CAC
:107650002BE4B24642E41B99002940F3E381129ED9
:107660000F9B9E42A8BF1E46002E0BDD229B0133BE
:107670003444072BC9E900562394229300F3AE83C8
:1076800009F108090F9F002EA8BFBF1B002F00F3B0
:1076900075811B9A129B9A4280F25381149B159913
:1076A0001C44C9E90013229B23940133072B229326
:1076B00000F3FB8209F10809129B0F999A1A5E1ACE
:1076C0009642A8BF1646002E0EDD229BC9F8046024
:1076D00001330D443444072BC9F8005023942293FE
:1076E00000F38B8309F10809002EACBF951B1546EA
:1076F000002D7FF7D1AB102D229B524E7FF7ADAE00
:10770000DDF830A0102705E009F10809103D102D23
:107710007FF7A3AE01331034072BC9E90067CDE929
:107720002234F1DD21AA5946504600F0B7FC00286A
:107730007FF491AEDDE922340DF1B809E6E7089A4D
:10774000002A40F02E83002308930A932EAD75E59E
:10775000069BD9073FF5A2AE0123072FCDE922747E
:10776000C9F80050C9F804307FF7C9AE0C9821AAB7
:10777000594600F093FC00287FF46DAEDDE92274D9
:107780000DF1B80ABBE6B9F1000F7FF7B8AEB9F159
:10779000100F2C4E40F3BE81CDF820801025DDF86F
:1077A000308007E00AF1080AA9F11009B9F1100FB9
:1077B00040F3AE8101371034072FCAE90065CDE9E7
:1077C0002274EFDD21AA5946404600F067FC0028EC
:1077D0007FF441AEDDE922740DF1B80AE4E70C98BC
:1077E00021AA594600F05AFC00287FF434AE239CAD
:1077F0000DF1B809FFF73DBB53422D21012222E4D0
:107800000C9821AA594600F049FC00287FF423AEC9
:10781000DDE922740DF1B80A4AE60C9821AA59460E
:1078200000F03CFC00287FF416AEDDE922740DF177
:10783000B80A4AE60D92FFF730BA2EADFEE400BF5B
:10784000648700007487000030228DF868208DF86E
:10785000697044F002040222FFF7F4BB12B213462F
:10786000FFF79DBBDDE9100102460B4600F020FD4D
:10787000002840F03E83089A27F02003511C0A9309
:1078800000F0B882472B00F0B280DDE9101244F41A
:10789000807306931346002BC0F221820793DDF814
:1078A00040A000230E93662F00F07481462F00F055
:1078B00071810A9B452B5246079B00F075821FA9D8
:1078C00004911CA903911BA9089E029102210C9806
:1078D00001960091FBF70CFC672F054640F04583AD
:1078E000E30700F173821F9B5B1B12931B9B0F939B
:1078F0000A9B472B40F09B810F9BDE1CC0F29681B8
:10790000089A9A42C0F29281129B0F9A934200F316
:10791000D682E4070F9B00F1FD8223EAE37207920F
:107920000A9367270E9B002B00F052822D238DF8BF
:10793000673000230893FFF71FBB01232B20FFF7BD
:10794000ACB9069BD8073FF5A9AE129B0F999A1ABE
:107950005B1A9342A8BF13461E46C5E60C98402109
:10796000FCF71EFECAF80000CAF81000002800F05C
:10797000FE824023CAF81430FFF760B9102F229B13
:10798000A64E40F38081324608955E460C9D4FF02E
:10799000100A934605E009F10809103F102F40F343
:1079A0006E8101331034072BC9E900BACDE92234C6
:1079B000F1DD21AA3146284600F070FB00287FF453
:1079C00048AEDDE922340DF1B809E6E72846CDF8E6
:1079D00020A00D960694F9F7D3FF20EAE0739DF8F6
:1079E00067100A900793CDF83CA0FFF7C2BA002AAF
:1079F000134608BF0123089347E7894E2EADA6FB27
:107A00000302D20802EB8200A3EB4000303005F8FD
:107A1000010D184609281346F1D82EAB5B1B0694BE
:107A20000A930BE4229B7F4AC9F8002001330134FA
:107A30000122072B23942293C9F8042000F34281EA
:107A400009F10809002971D1069B129A03F001037C
:107A500013433FF421AA149B15991A19C9E900137D
:107A6000229B23920133072B229300F3808109F19B
:107A700008091299C9F8005001338C18072BCDE979
:107A80002234C9F804107FF705AAF1E40C98179383
:107A900021AA594600F002FB00287FF4DCAC239CAD
:107AA000179B0DF1B809FFF7B1B9AA46FFF716BA4F
:107AB0000C9821AA594600F0F1FA00287FF4CBACCB
:107AC000239C0DF1B809FFF7DEBB0C9821AA59469B
:107AD00000F0E4FA00287FF4BEAC239C0DF1B80955
:107AE000FFF7BFB90C9821AA594600F0D7FA002831
:107AF0007FF4B1AC239C0DF1B809FFF7DABB062B7C
:107B000028BF0623484D0A930D960793FFF767B9E0
:107B1000DDF82080CAF8006001374C44072FCDE91A
:107B20002274CAF804907FF7E8AC1FE6149B1598FE
:107B30001A19C9E90003229B23920133072B2293D0
:107B400000F3158109F10809002992DA4F4210313A
:107B5000324E80F29381DDF830A0102405E009F167
:107B60000809103F102F40F3898101331032072B91
:107B7000C9E90064CDE92232F1DD21AA5946504617
:107B800000F08CFA00287FF466ACDDE922320DF1BA
:107B9000B809E6E71FA9DDE9073604911CA903919E
:107BA0001BA90291032101960C9800915246FBF704
:107BB0009FFA054686192B78302B00F08C811B9B91
:107BC0001E44079950460022002300F03FFB002886
:107BD00040F08C801F9BB34206D230215A1C1F926A
:107BE00019701F9B9E42F9D85B1B12931B9B0F932E
:107BF0000A9B472B3FF480AE662F18D1089A04F0F9
:107C0000010313430F9A002A40F3AA80002B40F08F
:107C100089810F9B07930A9384E600BF7487000055
:107C2000CDCCCCCC9884000090840000023F0F9A09
:107C30008DF87470531E002B1B93B6BFC2F1010365
:107C40002B222D22092B8DF8752055DC30338DF831
:107C5000773030238DF8763004231693129A169BD2
:107C6000012A13440A9340F321810A9B149A134476
:107C70000A9323EAE373079300230F9352E65A46CD
:107C8000089DB346164601333C44072BCDE9223408
:107C9000C9F80060C9F8047077DC09F10809F8E454
:107CA0002D218DF86710FFF756B90C9821AA594677
:107CB00000F0F4F900287FF4CEAB1B9A239C0DF161
:107CC000B809F9E40C9821AA594600F0E7F9002810
:107CD0007FF4C1AB1B99239C0DF1B809B2E603F107
:107CE000004307932D238A460E93DCE533467BE75A
:107CF0008DF86700FFF767B80DF18306DFF880C2E3
:107D0000324610468CFB0321DA17C2EBA10202EBCC
:107D10008201A3EB4101303100F8011C19466329AF
:107D2000134600F1FF32ECDC3033D9B2831E9E42A1
:107D300002F8011C40F2168113460DF1760201E0B3
:107D400013F8011B02F8011B9E42F9D10DF18503C6
:107D50000DF176021B1A13441DAA9B1A16937DE798
:107D6000002B40F0F480012307930A93DAE50C9886
:107D700021AA594600F092F900287FF46CABDDE9A6
:107D800022321B990DF1B809DEE60C9821AA59465A
:107D900000F084F900287FF45EAB239C0DF1B80954
:107DA00077E4069CFFF70DB908990C984E1C1FA9A3
:107DB00004911CA903911BA9029102210196009133
:107DC000FBF796F90546472F3FF48AAD2E44F8E6B7
:107DD0000E9B9DF867100893FFF7CBB80C9821AA6B
:107DE000594600F05BF900287FF435AB239C0DF178
:107DF000B80947E40623089347E50C9821AA594699
:107E000000F04CF900287FF426AB1B9A129B239CB0
:107E10009A1A0DF1B80967E4089B9DF867100D9652
:107E2000069407930A9308900F90FFF7A2B88DF875
:107E30006700FFF7F6B88DF86700FFF7D8B90C9820
:107E400021AA594600F02AF9FFF748B88DF86700D3
:107E5000FFF71BB98DF86700FFF752B88DF8670080
:107E6000FFF793B88DF86700FFF756B98DF86700F4
:107E7000FFF762B98DF86700FFF79AB901333A440A
:107E8000072BCDE92232C9F80060C9F804707FF7EA
:107E9000EEAD0C9821AA594600F000F900287FF4B5
:107EA000DAAADDE922320DF1B809E2E514F00102A7
:107EB0000F927FF4DAAE23EAE373079332E5149A64
:107EC000129B13440F9A0A93002A35DD23EAE373C9
:107ED0000793672726E5079950460022002300F004
:107EE000B5F900287FF46BAE089BC3F101031B9327
:107EF00066E6119B234D002BB8BF2D2124F0800393
:107F00000693A8BF9DF867101F4BB8BF8DF8671088
:107F1000FFF726B8149A13440A9323EAE3730793EE
:107F20006727FFE40F9B149A1344089A1A4422EA25
:107F3000E2730A920793F5E40F9B0A9AC3F10103D7
:107F40001A4422EAE2730A9207936727EAE4149B31
:107F50000133EAE70D9A52F8045B0D9245EAE575A4
:107F6000FEF79BBE0223169378E6089E2BE70C9A39
:107F70000C2313604FF0FF330993FEF7B8BF00BF27
:107F8000676666666084000064840000F8B50D468C
:107F90001446064610B1836B002B43D0B4F90C2075
:107FA000A369A360170790B21BD52369CBB1EDB2CB
:107FB00081042F4622D522686169D31A994229DDAE
:107FC0000133A1680139A160511C216015706269FB
:107FD0009A422AD0A389DB0701D50A2D25D038463D
:107FE000F8BD21463046FAF765FF20BBB4F90C20F6
:107FF000236990B2EDB281042F46DCD442F40052E2
:10800000A281226E616922F4005222662268D31A8C
:108010009942D5DC21463046FCF750F858B9226821
:108020000123CEE7FCF7D2F8B8E721463046FCF74B
:1080300045F80028D3D04FF0FF37D0E770B50B4D8F
:1080400084B0D5F8E05004461E4621B1A847431C31
:1080500006D004B070BD0A4601A9A847431CF8D158
:1080600000228A233260236004B070BD30080020F3
:1080700049B1FF2A02D80A70012070478A230360A1
:108080004FF0FF3070470846704700BF08B5062024
:10809000FDF74AF90120F8F75BF900BF2DE9F04F31
:1080A0009368166883B09246002B71D08B680A687B
:1080B00081460C46083643E0A38913F4906F2DD017
:1080C000D4E90410571A00EB400808EBD878781C64
:1080D0004FEA680828444045424684BF80464246ED
:1080E0005B0539D511464846FCF75AFA019000283D
:1080F0003CD03A462169F9F733FBA289019B22F46F
:10810000906242F08002A281D819A8EB0707A7600D
:10811000C4F8148023612060A8462F463A46594689
:10812000FEF7F6FADAF80810A3682268A3EB080352
:108130003A44491BA3602260CAF8081041B30836CC
:1081400056E902B598461F461046002DF7D0AB42BF
:10815000B2D9A8462F46E1E74846FEF76BFB034637
:108160000028D1D121694846FCF786F8A3890C2262
:1081700043F04003C9F800204FF0FF30A3810022F4
:108180000023CAF80820CAF8043003B0BDE8F08F15
:1081900000200023CAF8043003B0BDE8F08F00BF10
:1081A0004FF0FF3C06E000BF4FF0010C02E000BFC3
:1081B0004FF0010C4DF804CD4FEA410C7FEA6C5CA6
:1081C0004FEA430C18BF7FEA6C5C1BD001B050EA49
:1081D000410C0CBF52EA430C91EA030F02BF90EA34
:1081E000020F0020704710F1000F91EA030F58BFF3
:1081F000994208BF90422CBFD8176FEAE37040F055
:10820000010070474FEA410C7FEA6C5C02D150EAF2
:10821000013C07D14FEA430C7FEA6C5CD6D152EAAD
:10822000033CD3D05DF8040B704700BF8446104672
:1082300062468C461946634600E000BF01B5FFF771
:10824000B7FF002848BF10F1000F01BD4DF808ED41
:10825000FFF7F4FF0CBF012000205DF808FB00BF12
:108260004DF808EDFFF7EAFF34BF012000205DF86C
:1082700008FB00BF4DF808EDFFF7E0FF94BF0120B9
:1082800000205DF808FB00BF4DF808EDFFF7CEFFBA
:1082900094BF012000205DF808FB00BF4DF808EDF9
:1082A000FFF7C4FF34BF012000205DF808FB00BFCA
:1082B0004FEA410C7FEA6C5C02D150EA013C0AD1E2
:1082C0004FEA430C7FEA6C5C02D152EA033C02D1D4
:1082D0004FF0000070474FF0010070474FEA410235
:1082E00012F5001215D211D56FF47873B3EB625208
:1082F00012D94FEAC12343F0004343EA505311F02F
:10830000004F23FA02F018BF404270474FF00000C0
:10831000704750EA013005D111F0004008BF6FF0FE
:10832000004070474FF00000704700BF024B5822DA
:108330001A604FF0FF3070472C0A0020024B582281
:108340001A604FF0FF3070472C0A00202E2E2F6845
:10835000616C2F7372632F68616C5F696F2E6300AD
:1083600045786974696E67207769746820737461F1
:108370007475732025642E0A002E2E2F68616C2FD1
:108380007372632F68616C5F6932635F6D5F7379CD
:108390006E632E63002E2E2F68616C2F7372632F15
:1083A00068616C5F75736172745F73796E632E635D
:1083B000002D2D2D204932432044657465637420BF
:1083C0002D2D2D2D0D0A0D0A0025635B324B002546
:1083D000635B750025635B3142002E2E2F68706C45
:1083E0002F736572636F6D2F68706C5F7365726356
:1083F0006F6D2E630000000000300040003400402C
:1084000000200141004001410000004300040043FE
:1084100000080043000C004303000000140020008B
:1084200000010000080900000000D700001BB70091
:10843000000000000000000000000000000000003C
:1084400000202020002025303278000D0A2530320F
:10845000783A00202D2D0000494E4600696E6600D6
:108460004E414E006E616E00303132333435363756
:108470003839414243444546000000003031323330
:108480003435363738396162636465660000000050
:10849000286E756C6C290000300000002020202020
:1084A000202020202020202020202020303030308C
:1084B0003030303030303030303030302A2A2A20DE
:1084C000627566666572206F766572666C6F77207E
:1084D0006465746563746564202A2A2A3A20746589
:1084E000726D696E617465640A000000496E6669A8
:1084F0006E697479000000004E614E0042616C6C40
:108500006F632073756363656564656400000000D4
:108510002F7661722F746D702F706F727461676542
:108520002F63726F73732D61726D2D6E6F6E652D7B
:10853000656162692F6E65776C69622D342E322E0B
:10854000302E32303231313233312F776F726B2F20
:108550006E65776C69622D342E322E302E323032B9
:1085600031313233312F6E65776C69622F6C6962FD
:10857000632F7374646C69622F64746F612E63007F
:108580002F7661722F746D702F706F7274616765D2
:108590002F63726F73732D61726D2D6E6F6E652D0B
:1085A000656162692F6E65776C69622D342E322E9B
:1085B000302E32303231313233312F776F726B2FB0
:1085C0006E65776C69622D342E322E302E32303249
:1085D00031313233312F6E65776C69622F6C69628D
:1085E000632F7374646C69622F6D707265632E63A0
:1085F00000000000000000000080E03779C3414324
:10860000176E05B5B5B89346F5F93FE9034F384DF8
:10861000321D30F94877825A3CBF737FDD4F1575A4
:10862000000000000000F03F0000000000002440B7
:1086300000000000000059400000000000408F4092
:10864000000000000088C34000000000006AF840FD
:108650000000000080842E4100000000D012634121
:108660000000000084D797410000000065CDCD4197
:10867000000000205FA00242000000E87648374278
:10868000000000A2941A6D42000040E59C30A24216
:108690000000901EC4BCD64200003426F56B0C438B
:1086A0000080E03779C3414300A0D8855734764332
:1086B00000C84E676DC1AB43003D9160E458E14393
:1086C000408CB5781DAF154450EFE2D6E41A4B4408
:1086D00092D54D06CFF08044F64AE1C7022DB5444D
:1086E000B49DD9794378EA440500000019000000E0
:1086F0007D0000002020202020202020202020207D
:1087000020202020303030303030303030303030A9
:10871000303030302C2066756E6374696F6E3A208D
:1087200000000000617373657274696F6E2022250A
:108730007322206661696C65643A2066696C652005
:10874000222573222C206C696E65202564257325F3
:10875000730A000043000000504F534958000000C6
:108760002E0000002020202020202020202020205B
:108770002020202030303030303030303030303039
:1087800030303030002020202020202020202828B9
:1087900028282820202020202020202020202020C1
:1087A0002020202020881010101010101010101001
:1087B0001010101010040404040404040404041031
:1087C00010101010101041414141414101010101BF
:1087D0000101010101010101010101010101010189
:1087E0001010101010104242424242420202020295
:1087F0000202020202020202020202020202020259
:108800001010101020000000000000000000000008
:108810000000000000000000000000000000000058
:108820000000000000000000000000000000000048
:108830000000000000000000000000000000000038
:108840000000000000000000000000000000000028
:108850000000000000000000000000000000000018
:108860000000000000000000000000000000000008
:1088700000000000000000000000000000000000F8
:108880000000000000000000F8B500BFF8BC08BC04
:108890009E467047CD020000F8B500BFF8BC08BC8A
:0888A0009E467047A50200008E
:1088A800080000200000000000000000F402002082
:1088B80058030020BC030020000000000000000056
:1088C80000000000000000000000000000000000A0
:1088D8000000000000000000000000000000000090
:1088E8000000000000000000000000000000000080
:1088F8000000000000000000000000000000000070
:10890800000000000000000000000000000000005F
:10891800000000000000000000000000000000004F
:10892800000000000000000000000000000000003F
:10893800000000000000000000000000000000002F
:10894800000000000000000000000000000000001F
:1089580001000000000000000E33CDAB34126DE6BC
:10896800ECDE05000B000000000000000000000025
:1089780000000000000000000000000000000000EF
:1089880000000000000000000000000000000000DF
:1089980000000000000000000000000000000000CF
:1089A80000000000000000000000000000000000BF
:108CC8000000000000000000200400202004002014
:108CD800280400202804002030040020300400204C
:108CE80038040020380400204004002040040020FC
:108CF80048040020480400205004002050040020AC
:108D0800580400205804002060040020600400205B
:108D1800680400206804002070040020700400200B
:108D280078040020780400208004002080040020BB
:108D3800880400208804002090040020900400206B
:108D48009804002098040020A0040020A00400201B
:108D5800A8040020A8040020B0040020B0040020CB
:108D6800B8040020B8040020C0040020C00400207B
:108D7800C8040020C8040020D0040020D00400202B
:108D8800D8040020D8040020E0040020E0040020DB
:108D9800E8040020E8040020F0040020F00400208B
:108DA800F8040020F8040020000500200005002039
:108DB80008050020080500201005002010050020E7
:108DC8001805002018050020200500202005002097
:108DD8002805002028050020300500203005002047
:108DE80038050020380500204005002040050020F7
:108DF80048050020480500205005002050050020A7
:108E08005805002058050020600500206005002056
:108E18006805002068050020700500207005002006
:108E280078050020780500208005002080050020B6
:108E38008805002088050020900500209005002066
:108E48009805002098050020A0050020A005002016
:108E5800A8050020A8050020B0050020B0050020C6
:108E6800B8050020B8050020C0050020C005002076
:108E7800C8050020C8050020D0050020D005002026
:108E8800D8050020D8050020E0050020E0050020D6
:108E9800E8050020E8050020F0050020F005002086
:108EA800F8050020F8050020000600200006002034
:108EB80008060020080600201006002010060020E2
:108EC8001806002018060020200600202006002092
:108ED8002806002028060020300600203006002042
:108EE80038060020380600204006002040060020F2
:108EF80048060020480600205006002050060020A2
:108F08005806002058060020600600206006002051
:108F18006806002068060020700600207006002001
:108F280078060020780600208006002080060020B1
:108F38008806002088060020900600209006002061
:108F48009806002098060020A0060020A006002011
:108F5800A8060020A8060020B0060020B0060020C1
:108F6800B8060020B8060020C0060020C006002071
:108F7800C8060020C8060020D0060020D006002021
:108F8800D8060020D8060020E0060020E0060020D1
:108F9800E8060020E8060020F0060020F006002081
:108FA800F8060020F806002000070020000700202F
:108FB80008070020080700201007002010070020DD
:108FC800180700201807002020070020200700208D
:108FD800280700202807002030070020300700203D
:108FE80038070020380700204007002040070020ED
:108FF800480700204807002050070020500700209D
:10900800580700205807002060070020600700204C
:1090180068070020680700207007002070070020FC
:1090280078070020780700208007002080070020AC
:10903800880700208807002090070020900700205C
:109048009807002098070020A0070020A00700200C
:10905800A8070020A8070020B0070020B0070020BC
:10906800B8070020B8070020C0070020C00700206C
:10907800C8070020C8070020D0070020D00700201C
:10908800D8070020D8070020E0070020E0070020CC
:10909800E8070020E8070020F0070020F00700207C
:1090A800F8070020F807002000080020000800202A
:1090B80008080020080800201008002010080020D8
:1090C8001808002018080020FFFFFFFF000002001A
:1090D8004300000000000000000000000000000045
:1090E8000000000000000000000000000000000078
:1090F8004300000000000000000000000000000025
:109108000000000000000000000000000000000057
:109118004300000000000000000000000000000004
:109128000000000000000000000000000000000037
:1091380043000000000000000000000000000000E4
:109148000000000000000000000000000000000017
:1091580043000000000000000000000000000000C4
:1091680000000000000000000000000000000000F7
:1091780043000000000000000000000000000000A4
:1091880000000000000000000000000000000000D7
:109198004300000000000000000000000000000084
:1091A80000000000000000000000000000000000B7
:1091B80071800000E5660000000000008487000060
:1091C80060870000208700002087000020870000BB
:1091D80020870000208700002087000020870000EB
:1091E8002087000020870000FFFFFFFFFFFFFFFF31
:1091F800FFFFFFFFFFFF0000010041534349490003
:109208000000000000000000000000000000000056
:1092180000000000000000000000415343494900DD
:109228000000000000000000000000000000000036
:0C9238000000000000000000000000002A
:00000001FF
